:020000040000FA
:040200006BEF03F0AD
:040208000EEF01F004
:080218002DEF01F0D8CF01F039
:10022000E0CF02F0006EF3CF03F0F4CF04F0F0ACB7
:100230001DEF01F0F0B066EC0BF0A2A023EF01F08F
:10024000A1B018EC09F003C0F3FF04C0F4FF0050A4
:1002500002C0E0FF01C0D8FF1000D8CF06F0E8CF01
:1002600005F0E0CF07F0F3CF08F0F4CF09F0F0BCD1
:100270003DEF01F0F0B066EC0BF0A2B043EF01F0FF
:10028000A1B018EC09F0A2B04CEF01F0AECFE8FF3E
:100290006ECFE8FF52EF01F09EBA0CEC0FF0A4BA5B
:1002A00077EC0FF008C0F3FF09C0F4FF07C0E0FFD0
:0A02B00005C0E8FF06C0D8FF1000EB
:10030000F95000011150F926E4EF29F0E6EF29F049
:10031000F3EF29F008EF2AF016EF2AF024EF2AF085
:1003200032EF2AF040EF2AF050EF2AF05EEF2AF089
:100330006CEF2AF012000009D8A4A5EF01F000012B
:10034000000E0F6E000E106E1200E806030B0A0D71
:10035000F9CFE8FFF350F92683C00FF084C010F006
:10036000120085C00FF086C010F0120087C00FF099
:1003700088C010F0120089C00FF08AC010F012007F
:10040000EFCFE8FFE806070B0A0DF9CFE8FFF3503E
:10041000F9263CC04EF03DC04FF012003AC04EF0FD
:100420003BC04FF012003EC04EF03FC04FF01200F4
:1004300040C04EF041C04FF0120042C04EF043C0E9
:100440004FF0120044C04EF045C04FF0120046C0BD
:100450004EF047C04FF0120048C04EF049C04FF078
:1004600012000F0B060DF9CFE8FFF350F926BBC2BF
:10047000E8FF1200BCC2E8FF1200BDC2E8FF120094
:10048000BEC2E8FF1200BFC2E8FF1200C0C2E8FF10
:100490001200C1C2E8FF1200C2C2E8FF1200C3C2CC
:1004A000E8FF1200C4C2E8FF1200C5C2E8FF120054
:1004B000C6C2E8FF1200C7C2E8FF1200C8C2E8FFC8
:0E04C0001200C9C2E8FF1200CAC2E8FF120013
:100500000001E806070B0A0DF9CFE8FFF350F926C2
:100510008D510D6E8E510E6E12008F510D6E9051D9
:100520000E6E120091510D6E92510E6E120093518B
:100530000D6E94510E6E120095510D6E96510E6E09
:10054000120097510D6E98510E6E120099510D6E5A
:100550009A510E6E12009B510D6E9C510E6E120040
:100600000001E8BE33EF03F0E806070B0A0DF9CF4F
:10061000E8FFF350F9260D5073270E507423120093
:100620000D5075270E50762312000D5077270E506F
:10063000782312000D5079270E507A2312000D50A6
:100640007B270E507C2312000D507D270E507E23F9
:1006500012000D507F270E50802312000D5081276D
:100660000E5082231200E806070B0A0DF9CFE8FFAF
:10067000F350F9260D50736F0E50746F12000D5029
:10068000756F0E50766F12000D50776F0E50786FA9
:1006900012000D50796F0E507A6F12000D507B6F63
:1006A0000E507C6F12000D507D6F0E507E6F120049
:1006B0000D507F6F0E50806F12000D50816F0E50E5
:1006C000826F1200F2AE12000001010EA16FA1674D
:1006D00067EF03F0120092988098939C819C000130
:1006E0005B6A5C6A640E9DEC0BF092988098000146
:1006F000546A640E9DEC0BF00F018350306E316E26
:10070000326E0F018450336E346E356E0F01999046
:10071000878094969394829681940001000E176EC0
:10072000000E186E0001000E196E000E1A6E000108
:10073000000E1B6E000E1C6E0001000E1D6E000EE2
:100740001E6E0001000E136E000E146E0001000EEE
:10075000156E000E166E0001000EAB6F000EAC6F32
:100760000001000EAD6F000EAE6F0001000EAF6F06
:10077000000EB06F0001000EB16F000EB26F0001ED
:100780005E6A5F6A606BA16BA26BA36BE769E96B42
:100790000201BA6B0101116B0001CC6B4EEC32F01F
:1007A000020100510001A56F040E93EC08F0040E45
:1007B00093EC08F00001C350C56FC450C66F050E1E
:1007C00093EC08F0050E93EC08F00001C350C76FDE
:1007D000C450C86F000EE8CF0DF0E86AE8CF0EF005
:1007E000A8EC0BF0E8CF00F5010EE8CF0DF0E86AB9
:1007F000E8CF0EF0A8EC0BF0E8CF01F5C0EC0CF060
:10080000FA0E9DEC0BF0FA0E9DEC0BF0FA0E9DEC3F
:100810000BF0FA0E9DEC0BF0C8EC08F0C6EC24F0DF
:10082000A5EC0EF0B9EC0EF0F28EF28CD08E0F012A
:10083000D89083B6D880D8B023EF04F00A0E9DEC90
:100840000BF00F01D89083B6D880D8B039EF04F000
:100850000F01D89084B2D880D8B034EF04F00A0EDB
:100860009DEC0BF00F01D89084B2D880D8A05BEF3C
:1008700004F092EC1EF00201A50EA76346EF04F00F
:10088000E70EA86346EF04F04AEF04F04EEC32F0B6
:10089000C9EC0BF000C2E8FF0DEC1FF00301AD51F5
:1008A0000201A56FE9EC0AF064EC0AF00101F20E16
:1008B000066FA1EC0AF00F01D89084B2D880D8A0BE
:1008C0005BEF04F00A0E9DEC0BF00F01D89084B2A0
:1008D000D880D8A05BEF04F00F01D89084B4D88002
:1008E000D8B078EF04F00A0E9DEC0BF00F01D89011
:1008F00084B4D880D8B08EEF04F00F01D89083B6BE
:10090000D880D8B089EF04F00A0E9DEC0BF00F01EF
:10091000D89083B6D880D8A0BBEF07F00201A0C260
:100920000AF00201FF0E0AB0A56FA561FBEF04F00B
:100930000301A6A1DBEF04F00F0183BEDBEF04F09F
:10094000800E0FEC0DF0000EF86E660EF76E0C0EBA
:10095000F66E85EC0DF0C00E0FEC0DF0000EF86E8B
:10096000650EF76EB20EF66E85EC0DF00F01D890A5
:1009700084B4D880D8B0C2EF04F00A0E9DEC0BF01E
:100980000F01D89084B4D880D8B0B6EF04F00F012E
:10099000D89084B4D880D8A0C7EF04F00A0E9DEC9C
:1009A0000BF00F01D89084B4D880D8A0C7EF04F022
:1009B000C80E9DEC0BF00201D1B1E2EF04F0D1A31F
:1009C000FBEF04F0800E00019D6F65EC31F0D890D4
:1009D00035EC27F0D8B0F2EF04F00201FF0EA56F5E
:1009E000FBEF04F0E9EC0AF064EC0AF0A1EC0AF089
:1009F0000A0E9DEC0BF00001010E366EA3C252F000
:100A0000A4C253F00201A25100014D6E69EC23F023
:100A100065EC1FF0FCAE10EF05F00F01939481948C
:100A2000000133B030EF05F0010E366296EF05F0AD
:100A30000001050EE8CF5DF0070E37EC0AF0020E5C
:100A4000366E0001A5510201006329EF05F096EF13
:100A500005F0006F0DEC1FF065EC1FF096EF05F050
:100A6000010E366E0AEC23F0FDEC17F040EC07F0B7
:100A70000201A1A161EF05F00301B6517EEC24F063
:100A8000D8A061EF05F00201B76759EF05F0ABC0E0
:100A900073F0ACC074F0ADC075F0AEC076F0AFC00E
:100AA00077F0B0C078F0B1C079F0B2C07AF061EF01
:100AB00005F0F08CF086A290E868E8CFEEF067EFE2
:100AC00005F0F09CF086A280E86AE8CFEEF0020123
:100AD000A0B186EF05F02FEC17F0D8B486EF05F043
:100AE000BCEC19F04FEC19F089EC1BF01BEC1CF07E
:100AF0001AEC1AF09FEC21F0BDEC1FF0A7EC21F0EE
:100B000000EC1BF00001E9673CEC10F062EC03F034
:100B1000FCEC1CF05EEC0EF00001A26794EF05F017
:100B20000A0EA26FDEEC05F00AEF05F0800E0FEC66
:100B30000DF0000EF86E670EF76E3E0EF66E85EC49
:100B40000DF0C00E0FEC0DF0000EF86E650EF76E96
:100B5000B20EF66E85EC0DF081EC1EF0D8A0B3EF6E
:100B600005F040EC25F0FDEC17F0BCEC19F04FEC73
:100B700019F089EC1BF01BEC1CF01AEC1AF09FEC3E
:100B800021F0BDEC1FF0A7EC21F000EC1BF0FCEC19
:100B90001CF05EEC0EF00AEF05F00001100E0B6E7B
:100BA000C00E0FEC0DF0000EE16E030EE26EE6508B
:100BB00000EC0DF00B2ED7EF05F012000001840EB3
:100BC0000FEC0DF0200E00EC0DF00201520EA5BF4F
:100BD000200E000100EC0DF00601CE517EEC24F059
:100BE000410ED8A0200E00EC0DF00301B2517EECB6
:100BF00024F04D0ED8B02D0E00EC0DF00301B351D2
:100C00007EEC24F04D0ED8B02D0E00EC0DF003015B
:100C1000B4517EEC24F04D0ED8B02D0E00EC0DF04A
:100C2000200E00EC0DF0800E0FEC0DF0B9C20DF0AF
:100C3000BAC20EF00E6A0001640E0F6E000E106E46
:100C400067EC10F013C011F014C012F08BC00DF05F
:100C50008CC00EF013C20FF014C210F067EC10F04D
:100C60001450E8CF13F01550E8CF14F0156A0101C5
:100C700011B14BEF06F000011150135C12501458E3
:100C8000E8AE4BEF06F0C90E00015D6E050E37ECC5
:100C90000AF001011169000115EC0EF0200EE8CFF9
:100CA0000AF0300E25640AC025F0255000EC0DF046
:100CB000265000EC0DF02E0E00EC0DF0275000EC4D
:100CC0000DF00301B6517EEC24F0D8A071EF06F0D0
:100CD000800E0FEC0DF000C513F001C514F0EBEC25
:100CE0000DF00201B8AF8AEF06F0B86B000EE8CF46
:100CF0000DF0E86AE8CF0EF000C5E8FFB3EC0BF0AA
:100D0000010EE8CF0DF0E86AE8CF0EF001C5E8FF6C
:100D1000B3EC0BF069EC07F0D8B0B4EF06F07AEC66
:100D200007F0D8B0B4EF06F0CBEC24F0D8B0B4EFB5
:100D300006F09DEC23F00001A351E812D8A4B4EF13
:100D400006F00201A0A1B2EF06F0C00E0FEC0DF00C
:100D5000000EF86E650EF76ECC0EF66E85EC0DF09B
:100D6000B4EF06F0CDEC05F0000133B4CFEF06F0A0
:100D700035A4CFEF06F03594010E5D6E050E37EC0D
:100D80000AF000015466CEEF06F0542ABEC358F0B4
:100D9000BFC359F0CA6BCB6BCFEF06F0540600010E
:100DA00054A002EF07F0596602EF07F03B0E5A62BB
:100DB000E1EF06F0050E5D6E0A0E37EC0AF002EF69
:100DC00007F01E0E5A62ECEF06F0030E5D6E0A0E7F
:100DD00037EC0AF002EF07F00A0E5A62F7EF06F05E
:100DE000010E5D6E0A0E37EC0AF002EF07F0060EF8
:100DF0005A6002EF07F0010E5D6E0A0E37EC0AF042
:100E000002EF07F07F0E5A6E5650CE6F5750CF6FDD
:100E1000010E54622BEF07F058505910D8B41AEF56
:100E200007F05850CE6F5950CF6F000E0301BD63CD
:100E30002BEF07F0020E0301BD5DD8B427EF07F0DA
:100E40000001CA51CE6FCB51CF6F2BEF07F0E86A8C
:100E50000001CE6FCF6F00018B0E0FEC0DF0CF5164
:100E6000E8CF13F0146A156A166AE3EC0DF03A0E37
:100E700000EC0DF0CE51E8CF13F0E3EC0DF01200D2
:100E80000301C0517EEC24F0D8A066EF07F0030107
:100E9000000EC16563EF07F000017ABF66EF07F04F
:100EA0000301C15100010D6E0E6A00010A0E0F6EA2
:100EB000000E106E67EC10F07951135E7A51145CDD
:100EC000D8B066EF07F00001E76912000001E76B98
:100ED0001200D8900001CCAF1200C00E0FEC0DF044
:100EE000000EF86E660EF76E780EF66E85EC0DF05D
:100EF000D88012000D0E93EC08F00D0E93EC08F064
:100F000069C00DF06AC00EF0A9C20FF0AAC210F0BD
:100F100067EC10F000011450136E1550146E16504B
:100F2000156E166A15EC0EF00001255026100F0BF9
:100F3000D890D8B41200C00E0FEC0DF0000EF86E71
:100F4000660EF76E660EF66E85EC0DF0CB0E0FECAE
:100F50000DF00001255000EC0DF0265000EC0DF0D6
:100F60002E0E00EC0DF0275000EC0DF0285000EC98
:100F70000DF0D88012000F01D89084B4D880D8A08A
:100F8000BBEF07F00A0E9DEC0BF00F01D89084B474
:100F9000D880D8A0BBEF07F00F01D89083B6D880D7
:100FA000D8A0CCEF07F00A0E9DEC0BF00F01D89003
:100FB00083B6D880D8A0CCEF07F0800E0FEC0DF0F0
:100FC0000F018350A2EC0DF00F018450A2EC0DF044
:100FD000C00E0FEC0DF00F018650A2EC0DF00F01CA
:100FE0008750A2EC0DF00F01835082868184E8B017
:100FF0008296E8B281948098E8B48088320E9DECA5
:101000000BF00F01D89084B4D880D8B00DEF08F061
:101010000A0E9DEC0BF00F01D89084B4D880D8B0A4
:10102000DDEF07F00F01D89084B4D880D8A012EF7C
:1010300008F00A0E9DEC0BF00F01D89084B4D88014
:10104000D8A012EF08F0C00E0FEC0DF0000EF86EF5
:10105000650EF76E220EF66E85EC0DF000010D6A3E
:10106000800E0FEC0DF0000EF86E650EF76E580E48
:10107000F66E85EC0DF0870E0FEC0DF000010D50B3
:10108000AFEC0DF093EC08F08C0E0FEC0DF00F01AF
:10109000C4CFE8FFAFEC0DF00F01C3CFE8FFAFEC1A
:1010A0000DF0320E9DEC0BF00F01D89084B4D88077
:1010B000D8B060EF08F00A0E9DEC0BF00F01D8904D
:1010C00084B4D880D8B030EF08F00F01D89084B441
:1010D000D880D8A065EF08F00A0E9DEC0BF00F0148
:1010E000D89084B4D880D8A065EF08F000010D2A0C
:1010F0000C0E0D6430EF08F0DDEF07F00001136A0D
:10110000146A156A166A0A6E0B6A0A5093EC08F0A4
:101110000001C3501326C4501422D8B0152A0B2E38
:1011200085EF08F012000A6EA10EC06E000EC16EAF
:101130000AC0E8FF31EC02F0E8AEC188E89EE8445E
:10114000E844C26EC2800000C282C2B2A5EF08F0BD
:101150000001C3CF69F0C4CF6AF00AC0E8FF1200F3
:101160000F01C282C2B2B2EF08F00001C35069277A
:10117000C4506A23120093EC08F0B0EC08F0B0EC15
:1011800008F0B0EC08F000016A336A9F693312007E
:1011900000014C6A566A576A280EE8CF55F00001E4
:1011A000900E526E010E536E0001900E4E6E010EA7
:1011B0004F6E506A516A100E0001E8CF4DF0386A48
:1011C0003A6A3C6A3E6A406A426A446A466A486AC7
:1011D0004A6A080EE8CF39F0E8CF3BF0E8CF3DF09F
:1011E000E8CF3FF0E8CF41F0E8CF43F0E8CF45F05B
:1011F000E8CF47F0E8CF49F0E8CF4BF0979E858ED7
:10120000000152500F01E8CFBBFF010153500F0105
:10121000E8CFBCFF0A0E0F01E8CFBAFF0F01A08094
:101220000F019E900F01080EE8CFB1FFB1801200B0
:101230000001EEA1857E0201BAAF22EF09F08770AE
:101240002AEF09F00001E5B129EF09F087802AEFC4
:1012500009F087900001BBCFE8FF4E26BCCFE8FF26
:101260004F224EC0E8FFE8CFBBFF4FC0E8FFE8CFFA
:10127000BCFF0001E86A4C64A1EC09F000014C2AB3
:101280004CC0E8FFFE0B4D6057EF09F04C6A500E62
:10129000E8CF4EF050C0E8FF4E5EC30EE8CF4FF0EF
:1012A00051C0E8FF4F5A506A516A9EEF09F04CA0B6
:1012B0006CEF09F052C0E8FFE8CF4EF053C0E8FFF2
:1012C000E8CF4FF0BAC2E8FF0001E5814C6298EF29
:1012D00009F0E59198EF09F0120E4C6284EF09F0E5
:1012E00050C0E8FFE8CF4EF051C0E8FFE8CF4FF024
:1012F0004F324E324F324E324F324E324F324E32EA
:101300000F0E4F1698EF09F0040EE8CFEAFF000E1B
:10131000E8CFE9FF4CC0E8FFE830E89EE804E926A2
:1013200000EC02F052C0E8FF4E5E53C0E8FF4F5A97
:101330004EC0E8FF50264FC0E8FF51220F01A19098
:10134000120093EC0EF09DEC0EF00001010E3662DF
:10135000B0EF09F000018286BDB18296FF0EBD6F2D
:1013600087900301CDBFB8EF09F0859EB9EF09F072
:10137000858E0001552EFFEF09F0C9EC24F0000125
:1013800054A0EFEF09F00001FF0EE763EFEF09F063
:1013900058C0E8FF5910D8B4E7EF09F05866D4EF09
:1013A00009F03C0E586E5906580658505A6E030103
:1013B000E86ABD11D8B4E7EF09F0000158505910A0
:1013C000D8B4E7EF09F0CA6BCB6BEFEF09F000017F
:1013D000CA2B3C0ECA63EFEF09F0CA6BCB2B280E69
:1013E000E8CF55F0562A3C0E5662FFEF09F0566AD8
:1013F000572A0501002BD8B4012B0201B86902015C
:10140000A1A108EF0AF0530EC5EC0EF00001A86B85
:10141000000183CFE8FF311AD8A4306E316E30C09E
:10142000E8FF3212000184CFE8FF341AD8A4336EEB
:10143000346E33C0E8FF351200015E665E065F66FB
:101440005F0660676007A167A107A267A207A3679D
:10145000A3075C662DEF0AF012005C2E1200807864
:101460005D4E12005BC0E8FFE8CF5CF01200E8CFF1
:101470005BF0E8CF5CF08088120000010ABE44EF08
:101480000AF0819E45EF0AF0818E828A829A0A468E
:101490000B2E3DEF0AF012000201AD510A6E080E4C
:1014A0000B6E3DEC0AF00201AC510A6E080E0B6E99
:1014B0003DEC0AF00201AB510A6E080E0B6E3DECDA
:1014C0000AF08686869612000BC113F00CC114F048
:1014D0000DC115F009C117F00AC118F06BEC11F03D
:1014E0000201A55101010F03F35000011326D8B0EA
:1014F000142AD8B0152A0101006B016B026B0001A0
:101500001350E846E846E880E8921F0B13B6E88ED1
:101510000101006F000113361436153613361436E8
:101520001536133614361536133614361536145050
:101530000101016F000115501F0B01011009026F1D
:10154000120064EC0AF0010108510A6E080E0B6EDD
:101550003DEC0AF0010107510A6E080E0B6E3DECDE
:101560000AF0010106510A6E080E0B6E3DEC0AF0FE
:1015700086868696010105510A6E080E0B6E3DECBB
:101580000AF0010104510A6E080E0B6E3DEC0AF0E0
:10159000010103510A6E080E0B6E3DEC0AF08686BF
:1015A0008696010102510A6E080E0B6E3DEC0AF0A0
:1015B000010101510A6E080E0B6E3DEC0AF00101AB
:1015C00000510A6E080E0B6E3DEC0AF08686869678
:1015D00012000F01939E949A939C819C819E829A03
:1015E000989686960201D1A118EF0BF0D1B318EFAF
:1015F0000BF004C206F105C207F106C208F101C2F0
:1016000003F102C204F103C205F10101700E0B6F78
:10161000C60E0C6F000E0D6F0101140E096F000E47
:101620000A6F01010E6B0A0E106F010E0F6F120090
:101630000201D1B13EEF0BF0D1A33EEF0BF00AC295
:1016400006F10BC207F10CC208F107C203F108C290
:1016500004F109C205F101016C0E0B6FCF0E0C6F86
:10166000000E0D6F0101640E096F000E0A6F01017B
:101670000E6B080E106F010E0F6F12000201D1B138
:1016800065EF0BF0D1B365EF0BF010C206F111C29C
:1016900007F112C208F10DC203F10EC204F10FC22C
:1016A00005F101014A0E0B6F190E0C6F010E0D6F43
:1016B00001010A0E096F000E0A6F01010B0E0E6F79
:1016C000320E106F020E0F6F1200120087B284EFFD
:1016D0000BF0D5AE76EF0BF0D6CFC1F0D7CFC2F07E
:1016E0000001C32BD8B4C42BF09012000001C351E9
:1016F000C411F090D8A41200E86AE8CFD7FFE8CF71
:10170000D6FFD58EF0901200F17AF0AC96EF0BF088
:101710000301CDA192EF0BF0F1AA859EF1BA858E5F
:1017200096EF0BF0F1AA858EF1BA859EF09012002B
:101730000000E82E98EF0BF012000A6EFA0E98ECFB
:101740000BF0FA0E98EC0BF00A2E9EEF0BF0120045
:101750000EC0E8FFAA6E0DC0E8FFA96EA69EA69C6B
:10176000A680A8501200A86E0EC0E8FFAA6E0DC099
:10177000E8FFA96EA69EA69CA684F29E550EA76EB3
:10178000AA0EA76EA682F28EA1A8C4EF0BF0A198B4
:101790001200800E0FEC0DF0000EF86E660EF76E64
:1017A0001E0EF66E85EC0DF0C00E0FEC0DF0000E67
:1017B000F86E650EF76EA00EF66E85EC0DF07EEC01
:1017C00027F0D8A009EF0CF0C00E0FEC0DF0000EC2
:1017D000F86E660EF76E300EF66E85EC0DF04EEC80
:1017E00032F0A7EC1EF00001600E9E6F00C2E8FF11
:1017F00038EC1FF00201002B0301072B3A0E0763A0
:1018000005EF0CF0062B300E076F00019E2FF6EF50
:101810000BF092EC1EF000C2E8FF0DEC1FF012007E
:1018200000011550F86E1450F76E1350F66E00015B
:101830000E50E26E0D50E16E0900F550E66E0A069C
:101840000900F550E66E0A2E1CEF0CF012000001A4
:101850001550F86E1450F76E1350F66EA68EA69CB7
:10186000A684A688F29E550EA76EAA0EA76EA68223
:101870000000F28E0001400E1326000E14221522E5
:101880000A2E27EF0CF0120062EC03F00001155055
:10189000F86E1450F76E1350F66EA68EA69CA684B2
:1018A000A688F29E550EA76EAA0EA76EA682F28E8D
:1018B0000A0000010E50E26E0D50E16E400E0B6EFC
:1018C000E6CFE8FFF56E0F000B2EFAD7A68EA69C8A
:1018D000A684F29E550EA76EAA0EA76EA682F28E61
:1018E000A6940001400E1326000E142215220001BA
:1018F000400E0D26000E0E220A2E44EF0CF01200B0
:1019000000011550F86E1450F76E1350F66EA68E47
:10191000A69CA684A688F29E550EA76EAA0EA76E58
:10192000A6820000F28E0A00080E0B6E00010E5017
:10193000E26E0D50E16E080E0C6EE6CFE8FFF56E1C
:101940000F000C2EFAD7A68EA69CA684F29E550EEA
:10195000A76EAA0EA76EA6820000F28E0B2EEBD702
:10196000A6940001400E1326000E14221522000139
:10197000400E0D26000E0E220A2E80EF0CF01200F3
:101980000F019A6A886A9396939A93988186818ABE
:101990008188140E9DEC0BF0380E0FEC0DF0050E47
:1019A0009DEC0BF0380E0FEC0DF0010E9DEC0BF0E2
:1019B000380E0FEC0DF0010E9DEC0BF0380E0FEC15
:1019C0000DF0060E0FEC0DF00E0E0FEC0DF0010EEB
:1019D0000FEC0DF0800E0FEC0DF0800E0FEC0DF003
:1019E000650EF76E340EF66E85EC0DF0C00E0FEC42
:1019F0000DF0650EF76E460EF66E85EC0DF01200DA
:101A00001EEC0DF032EC0DF0818A81980000000090
:101A100081860000000081960000000012001EEC8C
:101A20000DF032EC0DF0819A819800000000818663
:101A300000000000819600000000120025EC0DF06F
:101A4000D8B01EEF0DF09A6A12009A688188819AC8
:101A500000000000818600000000D89088B0D88087
:101A600081961200886AE8B08888E8B2888AE8B46B
:101A7000888CE8B6888EE8B88886E8BA8884E8BC9E
:101A80008882E8BE8880120010101010101010100C
:101A900018181818181818181C1C1C1C1C1C1C1CA6
:101AA0001E1E1E1E1E1E1E1E01010101010101013E
:101AB00003030303030303030707070707070707D6
:101AC0000F0F0F0F0F0F0F0F800E0FEC0DF00DC04B
:101AD000F6FF0EC0F7FFF86A85EC0DF01200C00E9D
:101AE0000FEC0DF00DC0F6FF0EC0F7FFF86A85ECA5
:101AF0000DF01200C00E0FEC0DF0CEC0F6FFCFC0FF
:101B0000F7FFF86A85EC0DF01200100E88EF0DF06B
:101B10000A6E0900F5CFE8FFE812D8B4A1EF0DF086
:101B200000EC0DF00A4EA1EF0DF00900F5CFE8FF33
:101B3000E812D8B4A1EF0DF000EC0DF00A2E89EFF9
:101B40000DF012000A6E080E0B6E300E0ABE310E3A
:101B500000EC0DF00A360B2EA5EF0DF012000A6E08
:101B60003A0E0B6E0AC0E8FFF00BE842E842E8428A
:101B7000E84230090B64070F00EC0DF00AC0E8FFE3
:101B80000F0B30090B64070F00EC0DF00AC0E8FFE3
:101B9000120015EC0EF0255000EC0DF0265000EC74
:101BA0000DF0275000EC0DF0285000EC0DF02950FE
:101BB00000EC0DF0120015EC0EF0CEEF0DF015EC70
:101BC0000EF0D1EF0DF015EC0EF0D4EF0DF015EC9A
:101BD0000EF0D7EF0DF015EC0EF0FFEC0DF02550E8
:101BE00000EC0DF0265000EC0DF0275000EC0DF04D
:101BF000285000EC0DF0295000EC0DF0120000010F
:101C0000300E25621200200E256E300E2662120064
:101C1000200E266E300E27621200200E276E300E28
:101C200028621200200E286E12000001196A1A6A3A
:101C3000100E176E270E186E6BEC11F0300E13108D
:101C4000256E1BC013F01CC014F01DC015F01EC083
:101C500016F0196A1A6AE80E176E030E186E6BEC0E
:101C600011F0300E1310266E1BC013F01CC014F0C0
:101C70001DC015F01EC016F0196A1A6A640E176EA0
:101C8000000E186E6BEC11F0300E1310276E1BC097
:101C900013F01CC014F01DC015F01EC016F0196A18
:101CA0001A6A0A0E176E000E186E6BEC11F0300EE9
:101CB0001310286E300E1B10296E12000001310E19
:101CC000376267EF0EF092EC1EF091EF0EF0320EDD
:101CD000376271EF0EF000C2E8FF0DEC1FF091EFDC
:101CE0000EF0330E376279EF0EF0A7EC1EF091EF95
:101CF0000EF0340E376281EF0EF000C2E8FF38ECD0
:101D00001FF0350E376291EF0EF00001FF0E0D6EE1
:101D1000030E0E6EE8CF0EF0FF0EB3EC0BF091EF5A
:101D20000EF0376A12000F01ABA21200AB98AB881D
:101D30000F01AE500001616B12000F016BA2120087
:101D40006B986B880F016E5012000C0EE8CFAFFF3E
:101D5000220EE8CFACFF900EE8CFABFF0001616B25
:101D60009F9A9D8A1200ACA2B3EF0EF0E8CFADFFB0
:101D70001200000EE8CF6FFF220EE8CF6CFF900E2E
:101D8000E8CF6BFFA59AA38A12006CA2C5EF0EF0F4
:101D9000E8CF6DFF1200E1CF21F0E2CF22F0000189
:101DA00065C0E1FF000164C0E2FF686BACA2D6EF42
:101DB0000EF0E6CFE8FF00016827E8CFADFF000195
:101DC000662FD6EF0EF021C0E1FF22C0E2FF120025
:101DD000E1CF21F0E2CF22F0000165C0E1FF000178
:101DE00064C0E2FF686B0001050E5E6EE86A5E6427
:101DF00007EF0FF09EAAF7EF0EF0AECFE8FFE8CFA7
:101E0000E6FF000168270001662FF3EF0EF021C006
:101E1000E1FF22C0E2FF12009EAA12000001000EA4
:101E200061631FEF0FF0AECFE8FFE8CF62F0550E11
:101E300062631200280EE8CF5FF0612B1200010EE2
:101E4000616329EF0FF0AECFE8FFE8CF63F0612BBD
:101E50001200020E616333EF0FF0AECFE8FFE8CF60
:101E600064F0612B1200030E61633DEF0FF0AECF03
:101E7000E8FFE8CF65F0612B1200040E616346EFC6
:101E80000FF0AECFE8FFE8CF66F0612B050E61637F
:101E900052EF0FF0010E636350EF0FF0E8EC0EF01D
:101EA000612B1200060E616375EF0FF0AECFE8FFF5
:101EB000E8CF67F0020E636366EF0FF0CBEC0EF035
:101EC00068C0E8FFB3EC0EF0616B120068C0E8FF79
:101ED000676370EF0FF00C0EB3EC0EF0616B120045
:101EE0000D0EB3EC0EF0616B1200616B1200A4AA30
:101EF00012006ECFE8FF0201A1B1ABEF0FF0530A61
:101F0000D8A412000201A0A1120000010F0E741546
:101F10001009C5EC0EF073C0E8FFC5EC0EF000012F
:101F20000F0E76152009C5EC0EF07551C5EC0EF0BC
:101F300000010F0E78153009C5EC0EF07751C5EC95
:101F40000EF000010F0E7A154009C5EC0EF0795124
:101F5000C5EC0EF012000001A8B1B2EF0FF0AA6FAD
:101F6000A82B1200A96FA82B020EA863CBEF0FF0CD
:101F7000AA51F00B100AD8A410EF10F00F0EAA17F8
:101F8000AAA7C5EF0FF0F00EAA13A9C0ABF0AAC024
:101F9000ACF010EF10F0040EA863E2EF0FF0AA51BE
:101FA000F00B200AD8A410EF10F00F0EAA17AAA762
:101FB000DCEF0FF0F00EAA13A9C0ADF0AAC0AEF08E
:101FC00010EF10F0060EA863F9EF0FF0AA51F00B16
:101FD000300AD8A410EF10F00F0EAA17AAA7F3EF3B
:101FE0000FF0F00EAA13A9C0AFF0AAC0B0F010EF26
:101FF00010F0080EA86310EF10F0AA51F00B400A81
:10200000D8A410EF10F00F0EAA17AAA70AEF10F02D
:10201000F00EAA13A9C0B1F0AAC0B2F010EF10F0F0
:1020200012000C0E0F016F6E220E6C6E900EE8CF38
:102030006BFF12000001E80E0D26030E0E22780E33
:102040000D5C070E0E58D8A029EF10F0EF0E30EF00
:1020500010F00E320D320E320D320E320D320D50A6
:10206000C5EF0EF0BC0E0D5C030E0E58D8A02BEF82
:1020700010F0EF0E30EF10F0F00EC5EC0EF0800E09
:10208000C5EC0EF073C00DF074C00EF01AEC10F039
:1020900075C00DF076C00EF01AEC10F077C00DF0A0
:1020A00078C00EF01AEC10F079C00DF07AC00EF086
:1020B00032EC10F07BC00DF07CC00EF032EC10F072
:1020C0007DC00DF07EC00EF032EC10F0120078EC06
:1020D00010F010AE70EF10F00D50155E0E50165A45
:1020E0000EAE77EF10F00F50155E1050165A12001A
:1020F0000001136A146A156A166A0F500D02F3CFB5
:1021000013F0F4CF14F00F500E02F3501426F450D5
:102110001522D8B0162A10500D02F3501426F45090
:102120001522D8B0162A10500E02F3501526F4507E
:10213000162212000001246A1B6A14501310D8B42E
:10214000000C14501718E8BE241EA46B000E17AE26
:10215000ACEF10F0171E172A14AEB3EF10F0131ED9
:10216000141E132A142214501710E8BE3FEF11F06A
:1021700017501B5E143614341B3617501B261436AA
:1021800014341B36175014B01B5E14A01B261436D3
:1021900014341B36175014B01B5E14A01B261436C3
:1021A00014341B36175014B01B5E14A01B261436B3
:1021B00014341B36175014B01B5E14A01B261436A3
:1021C00014341B36175014B01B5E14A01B26143693
:1021D00014341B36175014B01B5E14A01B26143683
:1021E00013341B36175014B01B5E14A01B26133675
:1021F00013341B36175013B01B5E13A01B26133667
:1022000013341B36175013B01B5E13A01B26133656
:1022100013341B36175013B01B5E13A01B26133646
:1022200013341B36175013B01B5E13A01B26133636
:1022300013341B36175013B01B5E13A01B26133626
:1022400013341B36175013B01B5E13A01B26133616
:1022500013341B36175013B01B5E13A01B26133606
:1022600013A01B26A4B15DEF11F024AE000C131EC9
:10227000141EE86A132A14221B1E1B2A000C17AE18
:1022800058EF11F014BE54EF11F0E8CF9DF0135049
:10229000E8CF1BF01B9E133614361450E8CF13F012
:1022A0009D51146A35EF11F0136A132A146A000C59
:1022B000141E131EA42BB8EF10F01B2A17501B621C
:1022C00035EF11F01B6A000E132A142214AE35EFFD
:1022D00011F02388FF0C0001246A1C6A1B6A155048
:1022E00014101310D8B4000C15501818E8BE241E92
:1022F000A46B000E18AE81EF11F0171E181E172ADE
:10230000182215AE8AEF11F0131E141E151E132A83
:102310001422152215501810E8BE14EF13F01750B0
:102320001B5E18501C5A153615341B361C361750B8
:102330001B2618501C22153615341B361C36175018
:1023400015A0A8EF11F01B5E18501C5AABEF11F04E
:102350001B2618501C22153615341B361C361750F8
:1023600015A0B8EF11F01B5E18501C5ABBEF11F00E
:102370001B2618501C22153615341B361C361750D8
:1023800015A0C8EF11F01B5E18501C5ACBEF11F0CE
:102390001B2618501C22153615341B361C361750B8
:1023A00015A0D8EF11F01B5E18501C5ADBEF11F08E
:1023B0001B2618501C22153615341B361C36175098
:1023C00015A0E8EF11F01B5E18501C5AEBEF11F04E
:1023D0001B2618501C22153615341B361C36175078
:1023E00015A0F8EF11F01B5E18501C5AFBEF11F00E
:1023F0001B2618501C22153614341B361C36175059
:1024000015A008EF12F01B5E18501C5A0BEF12F0CB
:102410001B2618501C22143614341B361C36175039
:1024200014A018EF12F01B5E18501C5A1BEF12F08C
:102430001B2618501C22143614341B361C36175019
:1024400014A028EF12F01B5E18501C5A2BEF12F04C
:102450001B2618501C22143614341B361C361750F9
:1024600014A038EF12F01B5E18501C5A3BEF12F00C
:102470001B2618501C22143614341B361C361750D9
:1024800014A048EF12F01B5E18501C5A4BEF12F0CC
:102490001B2618501C22143614341B361C361750B9
:1024A00014A058EF12F01B5E18501C5A5BEF12F08C
:1024B0001B2618501C22143614341B361C36175099
:1024C00014A068EF12F01B5E18501C5A6BEF12F04C
:1024D0001B2618501C22143614341B361C36175079
:1024E00014A078EF12F01B5E18501C5A7BEF12F00C
:1024F0001B2618501C22143613341B361C3617505A
:1025000014A088EF12F01B5E18501C5A8BEF12F0CB
:102510001B2618501C22133613341B361C3617503A
:1025200013A098EF12F01B5E18501C5A9BEF12F08C
:102530001B2618501C22133613341B361C3617501A
:1025400013A0A8EF12F01B5E18501C5AABEF12F04C
:102550001B2618501C22133613341B361C361750FA
:1025600013A0B8EF12F01B5E18501C5ABBEF12F00C
:102570001B2618501C22133613341B361C361750DA
:1025800013A0C8EF12F01B5E18501C5ACBEF12F0CC
:102590001B2618501C22133613341B361C361750BA
:1025A00013A0D8EF12F01B5E18501C5ADBEF12F08C
:1025B0001B2618501C22133613341B361C3617509A
:1025C00013A0E8EF12F01B5E18501C5AEBEF12F04C
:1025D0001B2618501C22133613341B361C3617507A
:1025E00013A0F8EF12F01B5E18501C5AFBEF12F00C
:1025F0001B2618501C22133613B003EF13F017508C
:102600001B2618501C22A4B138EF13F024AE000C86
:10261000131E141E151E000E132A142215221B1E33
:102620001C1E1B2A1C22000C18AE32EF13F015BE24
:102630002DEF13F0E8CF9DF01450E8CF1CF01350AD
:10264000E8CF1BF01C9E143615361550E8CF13F05A
:102650009D51156A146A06EF13F0136A132A146A5F
:10266000156A000C151E141E131EA42B8FEF11F0FB
:102670001B2AE86A1C2217501B6206EF13F0185041
:102680001C6206EF13F01C6A1B6A000E132A142248
:10269000152215AE06EF13F02388FF0C1E6A1D6A83
:1026A0001C6A1B6A16341B361C361D361E36175024
:1026B0001B5E18501C5A19501D5A1A501E5AA46AF3
:1026C000A45B163616341B361C361D361E36A43750
:1026D000175016A077EF13F01B5E18501C5A1950B4
:1026E0001D5A1A501E5AE86AA45B80EF13F01B268D
:1026F00018501C2219501D221A501E22E86AA423C9
:10270000163616341B361C361D361E36A4371750A7
:1027100016A096EF13F01B5E18501C5A19501D5A44
:102720001A501E5AE86AA45B9FEF13F01B2618503C
:102730001C2219501D221A501E22E86AA4231636A4
:1027400016341B361C361D361E36A437175016A0FD
:10275000B5EF13F01B5E18501C5A19501D5A1A5031
:102760001E5AE86AA45BBEEF13F01B2618501C2209
:1027700019501D221A501E22E86AA4231636163458
:102780001B361C361D361E36A437175016A0D4EF44
:1027900013F01B5E18501C5A19501D5A1A501E5A1D
:1027A000E86AA45BDDEF13F01B2618501C221950B9
:1027B0001D221A501E22E86AA423163616341B3630
:1027C0001C361D361E36A437175016A0F3EF13F033
:1027D0001B5E18501C5A19501D5A1A501E5AE86A8E
:1027E000A45BFCEF13F01B2618501C2219501D226D
:1027F0001A501E22E86AA423163616341B361C36DD
:102800001D361E36A437175016A012EF14F01B5EAB
:1028100018501C5A19501D5A1A501E5AE86AA45BC7
:102820001BEF14F01B2618501C2219501D221A50A1
:102830001E22E86AA423163616341B361C361D36B3
:102840001E36A437175016A031EF14F01B5E185037
:102850001C5A19501D5A1A501E5AE86AA45B3AEFC6
:1028600014F01B2618501C2219501D221A501E222B
:10287000E86AA423163615341B361C361D361E3660
:10288000A437175016A050EF14F01B5E18501C5AB6
:1028900019501D5A1A501E5AE86AA45B59EF14F0D9
:1028A0001B2618501C2219501D221A501E22E86A9D
:1028B000A423153615341B361C361D361E36A43798
:1028C000175015A06FEF14F01B5E18501C5A1950CA
:1028D0001D5A1A501E5AE86AA45B78EF14F01B26A2
:1028E00018501C2219501D221A501E22E86AA423D7
:1028F000153615341B361C361D361E36A4371750B8
:1029000015A08EEF14F01B5E18501C5A19501D5A5A
:102910001A501E5AE86AA45B97EF14F01B26185051
:102920001C2219501D221A501E22E86AA4231536B3
:1029300015341B361C361D361E36A437175015A00D
:10294000ADEF14F01B5E18501C5A19501D5A1A5046
:102950001E5AE86AA45BB6EF14F01B2618501C221E
:1029600019501D221A501E22E86AA4231536153468
:102970001B361C361D361E36A437175015A0CCEF5B
:1029800014F01B5E18501C5A19501D5A1A501E5A2A
:10299000E86AA45BD5EF14F01B2618501C221950CE
:1029A0001D221A501E22E86AA423153615341B3640
:1029B0001C361D361E36A437175015A0EBEF14F049
:1029C0001B5E18501C5A19501D5A1A501E5AE86A9C
:1029D000A45BF4EF14F01B2618501C2219501D2282
:1029E0001A501E22E86AA423153615341B361C36ED
:1029F0001D361E36A437175015A00AEF15F01B5EC2
:102A000018501C5A19501D5A1A501E5AE86AA45BD5
:102A100013EF15F01B2618501C2219501D221A50B6
:102A20001E22E86AA423153615341B361C361D36C3
:102A30001E36A437175015A029EF15F01B5E18504D
:102A40001C5A19501D5A1A501E5AE86AA45B32EFDC
:102A500015F01B2618501C2219501D221A501E2238
:102A6000E86AA423153614341B361C361D361E3670
:102A7000A437175015A048EF15F01B5E18501C5ACC
:102A800019501D5A1A501E5AE86AA45B51EF15F0EE
:102A90001B2618501C2219501D221A501E22E86AAB
:102AA000A423143614341B361C361D361E36A437A8
:102AB000175014A067EF15F01B5E18501C5A1950E0
:102AC0001D5A1A501E5AE86AA45B70EF15F01B26B7
:102AD00018501C2219501D221A501E22E86AA423E5
:102AE000143614341B361C361D361E36A4371750C8
:102AF00014A086EF15F01B5E18501C5A19501D5A71
:102B00001A501E5AE86AA45B8FEF15F01B26185066
:102B10001C2219501D221A501E22E86AA4231436C2
:102B200014341B361C361D361E36A437175014A01D
:102B3000A5EF15F01B5E18501C5A19501D5A1A505B
:102B40001E5AE86AA45BAEEF15F01B2618501C2233
:102B500019501D221A501E22E86AA4231436143478
:102B60001B361C361D361E36A437175014A0C4EF72
:102B700015F01B5E18501C5A19501D5A1A501E5A37
:102B8000E86AA45BCDEF15F01B2618501C221950E3
:102B90001D221A501E22E86AA423143614341B3650
:102BA0001C361D361E36A437175014A0E3EF15F05F
:102BB0001B5E18501C5A19501D5A1A501E5AE86AAA
:102BC000A45BECEF15F01B2618501C2219501D2297
:102BD0001A501E22E86AA423143614341B361C36FD
:102BE0001D361E36A437175014A002EF16F01B5ED8
:102BF00018501C5A19501D5A1A501E5AE86AA45BE4
:102C00000BEF16F01B2618501C2219501D221A50CB
:102C10001E22E86AA423143614341B361C361D36D3
:102C20001E36A437175014A021EF16F01B5E185063
:102C30001C5A19501D5A1A501E5AE86AA45B2AEFF2
:102C400016F01B2618501C2219501D221A501E2245
:102C5000E86AA423143613341B361C361D361E3680
:102C6000A437175014A040EF16F01B5E18501C5AE2
:102C700019501D5A1A501E5AE86AA45B49EF16F003
:102C80001B2618501C2219501D221A501E22E86AB9
:102C9000A423133613341B361C361D361E36A437B8
:102CA000175013A05FEF16F01B5E18501C5A1950F6
:102CB0001D5A1A501E5AE86AA45B68EF16F01B26CC
:102CC00018501C2219501D221A501E22E86AA423F3
:102CD000133613341B361C361D361E36A4371750D8
:102CE00013A07EEF16F01B5E18501C5A19501D5A87
:102CF0001A501E5AE86AA45B87EF16F01B2618507C
:102D00001C2219501D221A501E22E86AA4231336D1
:102D100013341B361C361D361E36A437175013A02D
:102D20009DEF16F01B5E18501C5A19501D5A1A5070
:102D30001E5AE86AA45BA6EF16F01B2618501C2248
:102D400019501D221A501E22E86AA4231336133488
:102D50001B361C361D361E36A437175013A0BCEF89
:102D600016F01B5E18501C5A19501D5A1A501E5A44
:102D7000E86AA45BC5EF16F01B2618501C221950F8
:102D80001D221A501E22E86AA423133613341B3660
:102D90001C361D361E36A437175013A0DBEF16F075
:102DA0001B5E18501C5A19501D5A1A501E5AE86AB8
:102DB000A45BE4EF16F01B2618501C2219501D22AC
:102DC0001A501E22E86AA423133613341B361C360D
:102DD0001D361E36A437175013A0FAEF16F01B5EEF
:102DE00018501C5A19501D5A1A501E5AE86AA45BF2
:102DF00003EF17F01B2618501C2219501D221A50E1
:102E00001E22E86AA423133613341B361C361D36E3
:102E10001E36A437175013A019EF17F01B5E185079
:102E20001C5A19501D5A1A501E5AE86AA45B22EF08
:102E300017F01B2618501C2219501D221A501E2252
:102E4000E86AA423133613B02EEF17F017501B2691
:102E500018501C2219501D221A501E22000C0F015E
:102E6000D89083B6D880D8B03BEF17F00A0E9DEC0F
:102E70000BF00F01D89083B6D880D8B0B1EF17F01F
:102E80000F01D89084B2D880D8B04CEF17F00A0E5A
:102E90009DEC0BF00F01D89084B2D880D8B0B1EF80
:102EA00017F00001CC6773EF17F00001CC69030144
:102EB00032C30DF033C30EF00001E80E0F6E030EA7
:102EC000106E67EC10F014C01CF115C01DF1030169
:102ED000345101011C270301355101011D2334C365
:102EE0001AF135C31BF1B4EC29F0D8B084EF17F018
:102EF000D8A48BEF17F001011A07D8A01B071A07F7
:102F0000D8A01B078BEF17F001011A2BD8B41B2B8D
:102F10001A2BD8B41B2B1CC10DF01DC10EF00101E2
:102F20001A5100010D5E01011B5100010E5A0001F2
:102F3000000E0F6E010E106E67EC10F00001E80E2F
:102F4000176E030E186E6BEC11F013C032F314C041
:102F500033F31AC134F31BC135F31AEC1AF0D884D9
:102F600012000001CC67B7EF17F0D8941200CC6BB9
:102F700082EC1FF0D894120000016951E8CF0DF0E7
:102F80006A51E8CF0EF06D510D5E6E510E5AD8A009
:102F9000D9EF17F06B51E8CF0FF06C51E8CF10F07C
:102FA00067EC10F01450E8CF71F01550E8CF72F0D4
:102FB00012006F51E8CF0FF07051E8CF10F067ECBE
:102FC00010F01450E8CF71F01550E8CF72F01200F5
:102FD00069C00DF06AC00EF06D510D5E6E510E5A53
:102FE0006BC00FF06CC010F067EC10F01450E8CF1D
:102FF00071F01550E8CF72F01200040E93EC08F057
:10300000040EBBEC08F015C26BF016C26CF017C2D0
:103010006DF018C26EF019C26FF01AC270F0BCECFD
:1030200017F071C034F172C035F171C073F072C025
:1030300074F0050E93EC08F0050EBBEC08F01BC213
:103040006BF01CC26CF01DC26DF01EC26EF01FC290
:103050006FF020C270F0BCEC17F071C036F172C096
:1030600037F171C075F072C076F0060E93EC08F07F
:10307000060EBBEC08F021C26BF022C26CF023C23A
:103080006DF024C26EF025C26FF026C270F0BCEC69
:1030900017F071C038F172C039F171C077F072C0A9
:1030A00078F0070E93EC08F0070E93EC08F027C2B7
:1030B0006BF028C26CF029C26DF02AC26EF0E8EC09
:1030C00017F071C03AF172C03BF171C079F072C073
:1030D0007AF0030E93EC08F000010F01C3CFE8FF74
:1030E000E8CF8BF0C4CFE8FFE8CF8CF0080E93EC6C
:1030F00008F02DC26DF02EC26EF02BC26BF02CC208
:103100006CF0E8EC17F071C083F072C084F0090E27
:1031100093EC08F031C26DF032C26EF02FC26BF04A
:1031200030C26CF0E8EC17F071C085F072C086F028
:103130000A0E93EC08F035C26DF036C26EF033C261
:103140006BF034C26CF0E8EC17F071C087F072C01D
:1031500088F00B0E93EC08F039C26DF03AC26EF0B5
:1031600037C26BF038C26CF0E8EC17F071C089F030
:1031700072C08AF00301B5517EEC24F0D8A0C8EFEC
:1031800018F00001E80E7B6F030E7C6FCDEF18F096
:103190000001180E7B6FFC0E7C6F000E93EC08F0A4
:1031A0003BC26BF03CC26CF03DC26DF03EC26EF0B3
:1031B000E8EC17F071C07DF072C07EF0010E93EC68
:1031C00008F03FC26BF040C26CF041C26DF042C2E9
:1031D0006EF0E8EC17F071C07FF072C080F0030170
:1031E000B7517EEC24F0D8A0FDEF18F00001E80EF6
:1031F000816F030E826F17EF19F00301B9517EEC56
:1032000024F0D8A00BEF19F00001180E816FFC0E0E
:10321000826F17EF19F00301B8517EEC24F0D8A0AB
:1032200017EF19F00001000E816F000E826F12007F
:103230000001106A0FBE101E67EC10F00001640E52
:10324000176E000E186E6BEC11F013C011F014C065
:1032500012F013C00FF014C010F00EAE35EF19F0DD
:103260000F1E101E0F2AD8B0102A67EC10F00001B4
:103270000A0E176E000E186E6BEC11F00B50E8CFB3
:1032800017F0186A17BE181E6BEC11F011500D5E86
:1032900012500E5A13500D2614500E221200030124
:1032A000AE517EEC24F073C00DF074C00EF0D8A0C7
:1032B00065EF19F003011B510001E8CF0FF0030186
:1032C0001751E8CF0BF06DEF19F003011A5100010F
:1032D000E8CF0FF0640EE8CF0BF018EC19F00DC03A
:1032E00073F00EC074F00301AF517EEC24F075C092
:1032F0000DF076C00EF0D8A089EF19F00301265129
:103300000001E8CF0FF003012251E8CF0BF091EF5D
:1033100019F0030125510001E8CF0FF0640EE8CF4A
:103320000BF018EC19F00DC075F00EC076F003012B
:10333000B0517EEC24F077C00DF078C00EF0D8A02C
:10334000ADEF19F0030131510001E8CF0FF0030197
:103350002D51E8CF0BF0B5EF19F00301305100010A
:10336000E8CF0FF0640EE8CF0BF018EC19F00DC0A9
:1033700077F00EC078F012000301AE517EEC24F01D
:10338000D8A0DBEF19F073C00FF074C010F017C3B2
:103390000DF018C30EF00E6A0DBE0E1E67EC10F095
:1033A0000001640E176E000E186E6BEC11F013C066
:1033B00073F014C074F00301AF517EEC24F0D8A078
:1033C000FAEF19F075C00FF076C010F022C30DF0BF
:1033D00023C30EF00E6A0DBE0E1E67EC10F0000146
:1033E000640E176E000E186E6BEC11F013C075F0C2
:1033F00014C076F00301B0517EEC24F0D8A019EF90
:103400001AF077C00FF078C010F02DC30DF02EC366
:103410000EF00E6A0DBE0E1E67EC10F00001640E79
:10342000176E000E186E6BEC11F013C077F014C01D
:1034300078F012000201B2519BEC01F00301A75198
:1034400000010F260301A8510001102218C30DF03E
:1034500019C30EF000010E6AFF0E0DBE0E6E67EC72
:1034600010F00001640E176E186A196A1A6A6BEC84
:1034700011F000010301195100010D6E0E6A0DBE1D
:103480000E1E0D360E360D5013260E5014221350FC
:103490007327145074230201B3519BEC01F0030114
:1034A000A95100010F260301AA510001102223C3D4
:1034B0000DF024C30EF000010E6AFF0E0DBE0E6E5D
:1034C00067EC10F00001640E176E186A196A1A6A28
:1034D0006BEC11F000010301245100010D6E0E6A26
:1034E0000DBE0E1E0D360E360D5013260E50142234
:1034F00013507527145076230201B4519BEC01F050
:103500000301AB5100010F260301AC510001102251
:103510002EC30DF02FC30EF000010E6AFF0E0DBE7C
:103520000E6E67EC10F00001640E176E186A196ACF
:103530001A6A6BEC11F0000103012F5100010D6EAE
:103540000E6A0DBE0E1E0D360E360D5013260E5091
:10355000142213507727145078230201B5519BECA5
:1035600001F036C30DF037C30EF000010E6AFF0EF6
:103570000DBE0E6E67EC10F00001640E176E186A37
:10358000196A1A6A6BEC11F00301010E3763E0EF60
:103590001AF00001030E0E6E186EE80E0D6E176E17
:1035A00079510D5E7A510E5A196A1A6A13C00FF0DA
:1035B00014C010F067EC10F06BEC11F0FAEF1AF099
:1035C000020E3763FAEF1AF0000179510D6E7A514D
:1035D0000E6E13C00FF014C010F067EC10F0000175
:1035E000030EE8CF18F0E80EE8CF17F0196A1A6A50
:1035F0006BEC11F000011350792714507A2312005C
:1036000000010E6A08C40DF00DBE0E6800010A0E1E
:103610000F6E000E106E67EC10F0135073271450ED
:10362000742300010E6A09C40DF00DBE0E6800017E
:103630000A0E0F6E000E106E67EC10F01350752717
:103640001450762300010E6A0AC40DF00DBE0E68F8
:1036500000010A0E0F6E000E106E67EC10F0135092
:1036600077271450782300010E6A0BC40DF00DBEAD
:103670000E6800010A0E0F6E000E106E67EC10F05F
:103680001350792714507A2300010E6A0CC40DF0F0
:103690000DBE0E6800010A0E0F6E000E106E67EC74
:1036A00010F013507B2714507C2300010E6A0DC4C8
:1036B0000DF00DBE0E6800010A0E0F6E000E106EAA
:1036C00067EC10F013507D2714507E2300010E6A22
:1036D0000EC40DF00DBE0E6800010A0E0F6E000E36
:1036E000106E67EC10F013507F27145080230001F8
:1036F0000E6A0FC40DF00DBE0E6800010A0E0F6EAB
:10370000000E106E67EC10F01350812714508223C6
:10371000120000010A0E0D6E000E0E6E0301BB5169
:103720007EEC24F0D8A0D1EF1BF003014DAFA4EF45
:103730001BF04CC30FF0106A0FBE106867EC10F05E
:1037400013C073F014C074F003014FAFB3EF1BF05C
:103750004EC30FF0106A0FBE106867EC10F013C074
:1037600075F014C076F0030151AFC2EF1BF050C3E7
:103770000FF0106A0FBE106867EC10F013C077F0FE
:1037800014C078F0030153AFD1EF1BF052C30FF018
:10379000106A0FBE106867EC10F013C079F014C007
:1037A0007AF00301BC517EEC24F0D8A014EF1CF099
:1037B000030155AFE7EF1BF054C30FF0106A0FBEC3
:1037C000106867EC10F013C073F014C074F00301BC
:1037D00057AFF6EF1BF056C30FF0106A0FBE10681C
:1037E00067EC10F013C075F014C076F0030159AF08
:1037F00005EF1CF058C30FF0106A0FBE106867EC9D
:1038000010F013C077F014C078F003015BAF14EF31
:103810001CF05AC30FF0106A0FBE106867EC10F06E
:1038200013C079F014C07AF000017AAF1200E86A90
:10383000796F7A6F12000201A1B112000301B65133
:103840007EEC24F0D8A01200000160671200020193
:103850009F510001606F0201010EB66339EF1CF049
:10386000010E00015D6E050E37EC0AF0280E000116
:10387000606F73C00DF074C00EF0DCEC1CF0D8A4C7
:103880006FEF1CF00201B66748EF1CF002019E5179
:10389000000174BF56EF1CF00301192719AF60EF48
:1038A0001CF0D8A660EF1CF063EF1CF00301195F59
:1038B00019BF60EF1CF0D8A660EF1CF068EF1CF099
:1038C00019BF68EF1CF0640E1961196F6DEF1CF0E1
:1038D000640EE81EE82A1965196F82EC1FF075C0A6
:1038E0000DF076C00EF0DCEC1CF0D8A4A5EF1CF0B7
:1038F0000201B6677EEF1CF002019E51000176BF07
:103900008CEF1CF00301242724AF96EF1CF0D8A6FF
:1039100096EF1CF099EF1CF00301245F24BF96EF93
:103920001CF0D8A696EF1CF09EEF1CF024BF9EEF73
:103930001CF0640E2461246FA3EF1CF0640EE81EDB
:10394000E82A2465246F82EC1FF077C00DF078C060
:103950000EF0DCEC1CF0D8A4DBEF1CF00201B66723
:10396000B4EF1CF002019E51000178BFC2EF1CF0C1
:1039700003012F272FAFCCEF1CF0D8A6CCEF1CF003
:10398000CFEF1CF003012F5F2FBFCCEF1CF0D8A6A8
:10399000CCEF1CF0D4EF1CF02FBFD4EF1CF0640E62
:1039A0002F612F6FD9EF1CF0640EE81EE82A2F65F7
:1039B0002F6F82EC1FF0120000010EAEE5EF1CF03D
:1039C0000D1E0E1E0D2AD8B00E2AD8900E320D32C2
:1039D0000E66EFEF1CF0640E0D64F4EF1CF00001B6
:1039E000640E0D6E000E0E6E0D50E832E8321F0BA5
:1039F000D8740DC0E8FF12000001BD6B000174BF58
:103A00000EEF1DF011C30DF012C30EF073C00FF0D6
:103A100074C010F067EC10F018EF1DF015C30DF036
:103A200016C30EF073C00FF074C010F067EC10F006
:103A300013C30DF014C30EF0000114500D261550E1
:103A40000E2262EC1EF00DC03CF00EC03DF00001F5
:103A500076BF37EF1DF01CC30DF01DC30EF075C00F
:103A60000FF076C010F067EC10F041EF1DF020C3AE
:103A70000DF021C30EF075C00FF076C010F067ECAA
:103A800010F01EC30DF01FC30EF0000114500D26E0
:103A900015500E2262EC1EF00DC03AF00EC03BF045
:103AA000000178BF60EF1DF027C30DF028C30EF0B2
:103AB00077C00FF078C010F067EC10F06AEF1DF0DF
:103AC0002BC30DF02CC30EF077C00FF078C010F0B0
:103AD00067EC10F029C30DF02AC30EF0000114505A
:103AE0000D2615500E2262EC1EF00DC03EF00EC0E9
:103AF0003FF032C30DF033C30EF079C00FF07AC03F
:103B000010F067EC10F034C30DF035C30EF0000177
:103B100014500D2615500E2262EC1EF00DC040F020
:103B20000EC041F03AC30DF03BC30EF07BC00FF066
:103B30007CC010F067EC10F03CC30DF03DC30EF0FC
:103B4000000114500D2615500E2262EC1EF00DC01F
:103B500042F00EC043F0D2EF1DF000017EBFBDEF7A
:103B60001DF01CC30DF01DC30EF07DC00FF07EC014
:103B700010F067EC10F0C7EF1DF020C30DF021C36B
:103B80000EF07DC00FF07EC010F067EC10F01EC389
:103B90000DF01FC30EF0000114500D2615500E221B
:103BA000E5EF1DF03EC30DF03FC30EF07DC00FF0FA
:103BB0007EC010F067EC10F040C30DF041C30EF072
:103BC000000114500D2615500E2262EC1EF00DC09F
:103BD00044F00EC045F012EF1EF0000180BFFDEF73
:103BE0001DF011C30DF012C30EF07FC00FF080C0A6
:103BF00010F067EC10F007EF1EF015C30DF016C3C0
:103C00000EF07FC00FF080C010F067EC10F013C30F
:103C10000DF014C30EF0000114500D2615500E22A5
:103C200025EF1EF042C30DF043C30EF07FC00FF02E
:103C300080C010F067EC10F044C30DF045C30EF0E7
:103C4000000114500D2615500E2262EC1EF00DC01E
:103C500046F00EC047F081C00DF082C00EF00EBEDF
:103C60003AEF1EF046C30FF047C310F067EC10F0B8
:103C700040EF1EF04AC30FF04BC310F067EC10F09A
:103C800048C30DF049C30EF00D5014260E501522F6
:103C900014C00DF015C00EF062EC1EF00DC048F01F
:103CA0000EC049F00001CC6761EF1EF00301B15175
:103CB0007EEC24F0D8A061EF1EF038C340F039C389
:103CC00041F012000201AE5100010D5C0201AF5142
:103CD00000010E58E8AE72EF1EF0AEC20DF0AFC29A
:103CE0000EF012000201B05100010D5C0201B15151
:103CF00000010E58E8BE1200B0C20DF0B1C20EF0C5
:103D00001200000133B490EF1EF035A490EF1EF0C6
:103D10003594010E5D6E050E37EC0AF0D880120066
:103D2000D89012000001000E0D6E020E0E6E000102
:103D3000000E136E000E146E010E156EE86A0A6E08
:103D400010EC0CF0020100510001A56F12000001FF
:103D5000000E0D6E020E0E6E0001000E136E000EB0
:103D6000146E010E156E040E0A6E44EC0CF0120077
:103D7000E846E8060B6E0001000E0D6E030E0E6E97
:103D80000001000E136E000E146E010E156E0B5026
:103D90001426E86A1522100E0A6E10EC0CF01200C0
:103DA000E846E8060B6E0001000E0D6E080E0E6E62
:103DB0000001000E136E000E146E010E156E0B50F6
:103DC0001426E86A1522400E0A6E10EC0CF0000171
:103DD000000EB56F030EB66F0001000EB36F030E39
:103DE000B46F0001080EB46F100EB76F56EC23F0DD
:103DF0000001000E0D6E080E0E6E0001000E136E17
:103E0000000E146E010E156E0B501426E86A152272
:103E1000010E0A6E44EC0CF01200E846E8060B6E48
:103E20000001000E0D6E030E0E6E0001000E136EEB
:103E3000000E146E010E156E0B501426E86A152242
:103E40000A6E10EC0CF00001000E0D6E040E0E6EEA
:103E50000001000E136E000E146E010E156E0B5055
:103E6000E82A1426E86A15220A6E10EC0CF01200FB
:103E7000E846E8060C6E0001000E0D6E030E0E6E95
:103E80000001000E136E000E146E010E156E0C5024
:103E90001426E86A1522040E0A6E44EC0CF00001A8
:103EA000000E0D6E040E0E6E0001000E136E000E5D
:103EB000146E010E156E0C50E82A1426E86A1522BD
:103EC000040E0A6E44EC0CF012000001000EB56FF7
:103ED000030EB66F0001000EB36F060EB46F000E36
:103EE000B76F56EC23F00001000EB56F040EB66FED
:103EF0000001000EB36F070EB46F000EB76F56ECE3
:103F000023F0120002010051E846E8060A6E0001A3
:103F1000000E0D6E030E0E6E0001000E136E000EED
:103F2000146E010E156E0A501426E86A1522010E51
:103F30000A6E44EC0CF0120073C08DF074C08EF069
:103F400075C08FF076C090F077C091F078C092F095
:103F500079C093F07AC094F07BC095F07CC096F065
:103F60007DC097F07EC098F07FC099F080C09AF035
:103F700081C09BF082C09CF012009CEC1FF00301FA
:103F8000B2517EEC24F0D8B0D8EF1FF0030EE26EF1
:103F90005C0EE16E76EC22F0610EE16E76EC22F0C2
:103FA000660EE16E76EC22F06B0EE16E76EC22F09E
:103FB0009CEC1FF00301B3517EEC24F0D8B0F9EF74
:103FC0001FF0030EE26E700EE16E76EC22F09CECB8
:103FD0001FF0750EE16E76EC22F09CEC1FF07A0E6D
:103FE000E16E76EC22F09CEC1FF07F0EE16E76EC39
:103FF00022F09CEC1FF00301B4517EEC24F0D8B009
:1040000014EF20F0030EE26E840EE16E76EC22F0E7
:10401000890EE16E76EC22F08E0EE16E76EC22F0E7
:10402000930EE16E76EC22F012008DC00DF08EC082
:104030000EF010C40FF000010EBE11C40FF0106A94
:104040000FBE106867EC10F00001640E176E000ED2
:10405000186E6BEC11F0000113C0E8FF912714C03B
:10406000E8FF922391C00DF092C00EF012C40FF041
:1040700000010EBE13C40FF0106A0FBE106867EC8B
:1040800010F00001640E176E000E186E6BEC11F04C
:10409000000113C0E8FF8D2714C0E8FF8E2391C0F4
:1040A0000DF092C00EF014C40FF000010EBE15C446
:1040B0000FF0106A0FBE106867EC10F00001640E7C
:1040C000176E000E186E6BEC11F0000113C0E8FFC4
:1040D0008F2714C0E8FF902393C00DF094C00EF01A
:1040E00016C40FF000010EBE106A0FBE106867EC18
:1040F00010F00001640E176E000E186E6BEC11F0DC
:10410000000113C0E8FF8F2714C0E8FF90238DC083
:1041100073F08EC074F08FC075F090C076F091C0CF
:1041200077F092C078F093C079F094C07AF00401EF
:1041300017A1A9EF20F08FC07DF090C07EF00401A0
:1041400018A1A9EF20F000017D1F7E1F7D2BD8B0A4
:104150007E2B030198A1C6EF20F08FC00DF090C018
:104160000EF091C00FF092C010F000010DC075F07C
:104170000EC076F00DC077F00EC078F00F507727A4
:10418000105078230F50755F1050765B030199A192
:10419000E3EF20F08FC00DF090C00EF08DC00FF057
:1041A0008EC010F000010DC075F00EC076F00DC08D
:1041B00073F00EC074F00F507327105074230F501B
:1041C000755F1050765B03019AA19EEF21F08DC0C0
:1041D0000DF08EC00EF00DC073F00EC074F00DC067
:1041E0007FF00EC080F00001640E176E000E186E96
:1041F00003019C51E812D8B447EF21F0E8BE25EF47
:1042000021F0640800010F6E106A74BF16EF21F0F0
:1042100073C00DF074C00EF067EC10F06BEC11F091
:1042200013C073F014C074F047EF21F000017FC099
:104230000DF080C00EF067EC10F06BEC11F013C0C5
:104240007FF014C080F047EF21F0640F00010F6E83
:10425000106A74AF3AEF21F073C00DF074C00EF025
:1042600067EC10F06BEC11F013C073F014C074F035
:1042700047EF21F000017FC00DF080C00EF067EC29
:1042800010F06BEC11F013C07FF014C080F003014C
:104290009BA151EF21F000017F1F801F7F2BD8B021
:1042A000802B0001640E176E000E186E03019D51E5
:1042B000E812D8B49EEF21F00301C651E812D8B439
:1042C00074EF21F00301C5517EEC24F0D8B09EEFCD
:1042D00021F00001E80E0D6E030E0E6E93510D5E7F
:1042E00094510E5A80EF21F00001E80E0D6E030E7E
:1042F0000E6E99510D269A510E22D8900E320D3223
:104300009DC30FF09EC310F0106A0FBE101E67EC25
:1043100010F06BEC11F01350732714507423030149
:104320009BB199EF21F00001131E141E132AD8B07F
:10433000142A000113507F27145080231200030118
:10434000A4A112009CEC1FF015EC20F01200030158
:10435000A4B1AFEF21F09CEC1FF015EC20F00301AD
:104360009EA1CAEF21F00301C2517EEC24F0D8A037
:10437000CAEF21F003019F5100010D6E0E6A00018A
:104380000A0E0F6E000E106E67EC10F013C079F07D
:1043900014C07AF00301A0A1F7EF21F00301C3518B
:1043A0007EEC24F0D8A0D9EF21F00301A151E2EF77
:1043B00021F00301C4517EEC24F0D8A0F7EF21F0E6
:1043C0000301A25100010D6E0E6A00010A0E0F6E6C
:1043D000000E106E67EC10F01350795D14507A598E
:1043E000E8AEF7EF21F013C079F014C07AF01200B4
:1043F0000BC0E8FFF00BD8B412000DC069F00EC07E
:104400006AF00EAE09EF22F00D1E0E1E0D2AD8B076
:104410000E2A0DC013F00EC014F0640E176E9AEC45
:1044200010F000011C6A090E136021EF22F00BC08E
:10443000E8FFE83AE8060F0BE8B63EEF22F033EF6C
:1044400022F0136E0DC01BF00EC01CF0840E000194
:104450001B5E030E1C5A0BC0E8FFE83AE8060F0B80
:10446000E8B63EEF22F00B0DF350460F1324E8CFD1
:10447000D9FF020EE8CFDAFF48EF22F0E8960B0DE5
:10448000F350DA0F1324E8CFD9FF030EE8CFDAFF99
:10449000DECF0AF0DFCF0BF000010BC00DF00AC039
:1044A000E8FF0D5E0E6A0DBE0E681BC00FF01CC04B
:1044B00010F067EC10F00A0E176E9AEC10F00AC0BC
:1044C000E8FF0A0DF3CFE8FF1326F4CFE8FF14222C
:1044D00013C00DF014C00EF000016AAF120000010D
:1044E0000D1E0E1E0D2AD8B00E2A1200E650E8CF7F
:1044F0000BF0E812D8B4120080EC02F0F8EC21F0D6
:104500000DC011F00EC012F0E6CF0AF0E6CFE8FFC2
:104510000001E8CF0DF00E6A0DBE0E1E00010A0E5E
:104520000F6E000E106E67EC10F011C00DF012C08F
:104530000EF013500D5E14500E5A0EBED5EF22F041
:10454000E6CFE8FF00010AACBEEF22F0E8CF13F09F
:10455000E9CF14F00DC011F00EC012F0135080EC32
:1045600002F00DC013F00EC014F00A0E176E9AEC94
:1045700010F011C00DF012C00EF013500F6E106A43
:104580000FBE101E67EC10F00001640E176E000ED7
:10459000186E196A1A6A6BEC11F013C00DF014C092
:1045A0000EF00A5000EC03F01200E6CFE8FFE6CF71
:1045B000E8FF00010AAAF3EF22F0E8CF13F00DC0E4
:1045C00011F00EC012F0135080EC02F00DC013F089
:1045D0000EC014F00A0E176E9AEC10F011C00DF018
:1045E00012C00EF013500F6E106A0FBE101E67EC53
:1045F00010F00001640E176E000E186E196A1A6A28
:104600006BEC11F013C00DF014C00EF00A5000EC6A
:1046100003F012000001BD0EB56F030EB66F00016E
:10462000120EB36F010EB46F050EB76F56EC23F088
:10463000D90EE8CFD9FF060EE8CFDAFF060EE8CF95
:104640000CF0DDCFE8FFE812D8B42EEF23F0DFCF77
:10465000E8FF7EEC24F0D8B03AEF23F0DDCFE8FF9E
:104660000C2E21EF23F0A5C0E8FF0201006343EF09
:1046700023F01200DECFE8FFDECFE8FF0201006387
:1046800043EF23F01200E8CF00F20DEC1FF0000121
:10469000120EB56F010EB66F0001BD0EB36F030EA3
:1046A000B46F050EB76F56EC23F012000001B55140
:1046B000E16EB651E26E0001B351D96EB451DA6EBB
:1046C000E6CFE8FFE8CFDEFF0001B72F60EF23F071
:1046D00012000001BF6B0301AE517EEC24F000011B
:1046E000D8B0BF810301AF517EEC24F00001D8B0F7
:1046F000BF830301B0517EEC24F00001D8B0BF8528
:104700000301B1517EEC24F00001D8B0BF87030152
:10471000B6517EEC24F00001D8B0BF890301BB5133
:104720007EEC24F00001D8B0BF8B0301BC517EECBD
:1047300024F00001D8B0BF8D1200C00E0FEC0DF0B8
:104740000301AE517EEC24F00001E86AE880BF1559
:10475000D8A0B9EF23F0D8A4CAEF23F0BF71000EA0
:10476000F86E660EF76E9C0EF66E85EC0DF07BEF24
:1047700024F0D8B0CAEF23F0D8B4CAEF23F0BF7149
:10478000000EF86E660EF76E8A0EF66E85EC0DF072
:104790007BEF24F00301AF517EEC24F00001E86AC6
:1047A000E882BF15D8A0E3EF23F0D8A4F4EF23F0FC
:1047B000BF73000EF86E660EF76EC00EF66E85ECD7
:1047C0000DF07BEF24F0D8B0F4EF23F0D8B4F4EF81
:1047D00023F0BF73000EF86E660EF76EAE0EF66E27
:1047E00085EC0DF07BEF24F00301B0517EEC24F05A
:1047F0000001E86AE884BF15D8A00DEF24F0D8A422
:104800001EEF24F0BF75000EF86E660EF76EE40E14
:10481000F66E85EC0DF07BEF24F0D8B01EEF24F09F
:10482000D8B41EEF24F0BF75000EF86E660EF76E5A
:10483000D20EF66E85EC0DF07BEF24F00301B15142
:104840007EEC24F00001D8A034EF24F0BFB735EFA0
:1048500024F0BF77000EF86E670EF76E2C0EF66E22
:1048600085EC0DF07BEF24F0BF970301B6517EEC91
:1048700024F00001D8A04BEF24F0BFB94CEF24F096
:10488000BF79000EF86E670EF76E1A0EF66E85ECA5
:104890000DF07BEF24F0BF990301BB517EEC24F0B7
:1048A0000001D8A062EF24F0BFBB63EF24F0BF7B10
:1048B000000EF86E660EF76EF60EF66E85EC0DF0D5
:1048C0007BEF24F0BF9B0301BC517EEC24F0000180
:1048D000D8A079EF24F0BFBD7AEF24F0BF7D000EA1
:1048E000F86E670EF76E080EF66E85EC0DF07BEF36
:1048F00024F0BF9D1200500EA36F1200E8AAAAEF89
:1049000024F0E8A8AAEF24F00A6E070BC90FE16EA5
:10491000030EE26EE65000010D6E0E6AE8BE0E68F0
:1049200000010A0E0F6E000E106E67EC10F00A50B8
:10493000070BE846340FE16E010EE252E650E6CF77
:104940000BF00001135E0B501458E8360ABE12003B
:10495000D8701200D890E8BA1200D880E8B81200D7
:1049600000011F6E206AE8BC2080070BE82AD8806F
:104970002036E82EB8EF24F030501FB63350201404
:10498000D8802062D8901FBED8701200040ED56E59
:104990001200D59E1200D89087B21200D880D5BEE2
:1049A0001200C3C00DF0C4C00EF000013C0E0F6E2B
:1049B000000E106E78EC10F013C00DF014C00EF065
:1049C0000001240E0F6EF40E106E78EC10F0C1C0D2
:1049D00017F0C2C018F00001000E196E000E1A6E1A
:1049E0004EEC13F0A5C317F0A6C318F00001186A27
:1049F0006BEC11F0C00E0FEC0DF0000EF86E650EB2
:104A0000F76EFA0EF66E85EC0DF0CB0E0FEC0DF096
:104A1000EBEC0DF0A5C313F0A6C314F0146AC00E9E
:104A20000FEC0DF0E7EC0DF00001000EC36F000E6F
:104A3000C46FD88012000001020E3662120000011D
:104A400033A01200FC6A0AEF05F034EC25F0D8A080
:104A50001200FC6AA7EC1EF000C2E8FF38EC1FF061
:104A600065EC1FF00AEF05F0000130B63EEF25F0CF
:104A700032A63EEF25F03296D8801200D890120070
:104A80000001670E0E6E500E0D6E87EC25F064EC83
:104A90000DF00001115080EC01F012001EC10DF06C
:104AA0001FC10EF064EC0DF012000001EF51D8B4FC
:104AB0001200E1CF3EF1E2CF3FF1FDEC17F0000133
:104AC000000E736F000E746F0001000E756F000E04
:104AD000766FBCEC19F04FEC19F089EC1BF01BEC75
:104AE0001CF01AEC1AF09FEC21F0BDEC1FF0A7ECC3
:104AF00021F000EC1BF0FCEC1CF05EEC0EF03EC173
:104B0000E1FF3FC1E2FF12000001EF6912001BEC60
:104B100025F00001CD6BDB6BEA6BEB6BC00E0FEC8D
:104B20000DF00DC0F6FF0EC0F7FFF86A0DC00FF0D4
:104B30000EC010F085EC0DF0FA0E9DEC0BF08EEC33
:104B400029F0D8A4AAEF25F0110E0D26D8B00E2A10
:104B5000B1EF25F0D8A0BEEF25F0130E0D26D8B08A
:104B60000E2A0DC0F6FF0EC0F7FFF86A0900F5CF58
:104B70000DF00900F5CF0EF08EEF25F025EC25F0B5
:104B800081EC1EF0D8A08EEF25F0150E0D26D8B0C2
:104B90000E2A0DC0F6FF0EC0F7FFF86A0900F5CF28
:104BA00011F00900F5CF12F00FC00DF010C00EF09B
:104BB0000900F5CF0FF00900F5CF10F00900F5CF8F
:104BC000CEF00900F5CFCFF00001B96BBA6BBB692D
:104BD0007F0EE8CFBCF012ACFAEF25F00900F5CF5C
:104BE000B9F00900F5CFBAF00900F5CFBBF0090024
:104BF000F5CFBCF012A403EF26F00900F5CFEAF0E0
:104C00000900F5CFEBF012A20CEF26F00900F5CF6A
:104C1000ECF00900F5CFEDF012AE11EF26F064ECE8
:104C20000DF012A616EF26F07AEC0DF012A212008B
:104C30000001E86AE8CFFBFFEDC0E8FFE8CFFAFF2C
:104C4000ECC0E8FFF96EE8CF0AF00FC01BF010C00F
:104C50001CF00FC0F6FF10C0F7FFF86A150EF6261D
:104C6000D8B0F72A0900F5CFE8FF0A6239EF26F03D
:104C700012000FC0F6FF10C0F7FF110EF626D8B0D5
:104C8000F72A0900F5CF0FF00900F5CF10F00FC09B
:104C9000E8FF1B6229EF26F010C0E8FF1C6229EF35
:104CA00026F01200000110500F10D8B41200E86A6C
:104CB000FB6E1050E8CFFAFF0F50F96E00010F5055
:104CC000E16E1050E26E0001000E11627CEF26F0E2
:104CD0000FC0F6FF10C0F7FFF86A160EF626D8B020
:104CE000F72ACEC0E1FFCFC0E2FFE7CFE8FF23EC19
:104CF00026F0FBEC28F01200010E116283EF26F083
:104D000025EC28F01200020E1162ADEF26F0000132
:104D100012A08EEF26F0CE510001B86FE6CF0AF058
:104D2000E5CF0BF000010AC011F00BC012F0129E8B
:104D3000129C7BEC28F000010FC0E1FF10C0E2FFE5
:104D400011C00AF012C00BF00AC0E6FFE7CFE8FF7F
:104D5000C00B0B120BC0E5FF1200030E1162C2EF75
:104D600026F0E7CFE8FFE8367EEC27F0000ED8B05B
:104D7000E81E0A6E00010FC0E1FF10C0E2FF0AC08A
:104D8000E7FF1200040E1162D3EF26F0E7CFE8FF31
:104D900042EC29F00A6E00010FC0E1FF10C0E2FFF3
:104DA0000AC0E7FF1200050E1162E5EF26F0E7CF1B
:104DB000E8FFD3EC27F0E8CF0AF000010FC0E1FFD5
:104DC00010C0E2FF0AC0E7FF1200060E1162FBEFFF
:104DD00026F0E7CF0AF00FC0CEF010C0CFF00001F0
:104DE000040E0F6E7B0E106E0AC0E8FF23EC26F057
:104DF000FBEC28F01200070E116202EF27F052ECD4
:104E000026F01200080E116213EF27F0E7CFE8FF3B
:104E1000CDEC27F0E8CF0AF000010FC0E1FF10C091
:104E2000E2FF0AC0E7FF0A0E116234EF27F0E7CF76
:104E3000E8FF0001CE15D890D8B4D8807EEC27F0DA
:104E40000001CEC00AF000010FC0E1FF10C0E2FF78
:104E5000D8B02FEF27F00AC0E8FFE71212000AC00F
:104E6000E8FFE81EE716120012000B6AD8B00B1E0E
:104E7000C00E0FEC0DF0000EF86E650EF76EA00E72
:104E8000F66E85EC0DF00BA05AEF27F0C80E0FEC74
:104E90000DF0280E00EC0DF0CC0E0FEC0DF0290EED
:104EA00000EC0DF0CF0E0FEC0DF0200E00EC0DF02D
:104EB0006CEF27F0C80E0FEC0DF0200E00EC0DF09B
:104EC000CC0E0FEC0DF0280E00EC0DF0CF0E0FEC19
:104ED0000DF0290E00EC0DF08EEC29F0D8B40B6A21
:104EE000FF0ED8B00B6E25EC25F081EC1EF0D8A09B
:104EF00043EF27F0D8900BB0D88012000B6AD8B0DF
:104F00000B1EC80E0FEC0DF0000EF86E650EF76E5E
:104F1000DE0EF66E85EC0DF00BA0A3EF27F0C80EA9
:104F20000FEC0DF0280E00EC0DF0CC0E0FEC0DF098
:104F3000290E00EC0DF0CF0E0FEC0DF0200E00EC62
:104F40000DF0B5EF27F0C80E0FEC0DF0200E00ECC1
:104F50000DF0CC0E0FEC0DF0280E00EC0DF0CF0E86
:104F60000FEC0DF0290E00EC0DF08EEC29F0D8B40A
:104F70000B6AFF0ED8B00B6E25EC25F081EC1EF00D
:104F8000D8A08CEF27F0D8900BB0D8801200000189
:104F9000BB65BB51B961B95112000001E86900015C
:104FA0009D6FD7EF27F000019D6F0001E86BC80EE1
:104FB0009DEC0BF09DC0E8FF0001136E146A156AAA
:104FC000166A15EC0EF00001E867F5EF27F0CD0E3C
:104FD0000FEC0DF0275000EC0DF0285000EC0DF018
:104FE000295000EC0DF004EF28F0CC0E0FEC0DF082
:104FF000275000EC0DF0285000EC0DF02E0E00ECC8
:105000000DF0295000EC0DF0B4EC29F00001D8A40B
:1050100010EF28F09D2BBB519D619D6F1BEF28F079
:10502000D8A01BEF28F09D51B9611BEF28F09D0718
:10503000B9519D659D6F25EC25F081EC1EF0D8A03F
:10504000D7EF27F000019D51120055EC25F0FA0E24
:105050009DEC0BF0E7CFE8FFE7BEE81EE7BEE82ACD
:105060000001136E146A156A166A15EC0EF0CB0E69
:105070000FEC0DF0200EE7BE2D0E00EC0DF02750CA
:1050800000EC0DF0285000EC0DF0295000EC0DF074
:10509000250E00EC0DF0B4EC29F00001D8A454EF7B
:1050A00028F0E72A58EF28F0D8A058EF28F0E706B4
:1050B00025EC25F081EC1EF0D8A025EF28F00001AA
:1050C000EF6B120000011150BB5D1250BC59D8B0FB
:1050D0006FEF28F0BB51116EBC51126E1200B95126
:1050E000115CBA511258D8B07AEF28F0B951116E4C
:1050F000BA51126E120062EC28F00001BE6B000182
:10510000B851E812D8B48DEF28F0B851E16E000E16
:10511000E26E11C0E6FF12C0E7FFF0C0E8FF7F08B3
:10512000E8BEE86AE8669DEC0BF011C013F012C00F
:1051300014F0D89014321332156A166A15EC0EF07A
:10514000C90E0FEC0DF0265000EC0DF02E0E00EC09
:105150000DF0275000EC0DF0285000EC0DF0295018
:1051600000EC0DF06D0E00EC0DF0530E00EC0DF0A8
:10517000B4EC29F00001D8A4CDEF28F0112AD8B45E
:10518000122A112AD8B4122ABC5112627BEF28F0DD
:10519000BB511160116E7BEF28F0D8A0DFEF28F033
:1051A0001106D8A012061106D8A01206BA51126232
:1051B0007BEF28F0B9511164116E7BEF28F00001EC
:1051C00033A2BE6933BCEAEF28F00001A00E116ED5
:1051D0000F0E126E000133BEF3EF28F00001D00E67
:1051E000116E070E126E25EC25F081EC1EF0D8A092
:1051F0007FEF28F01200C00E0FEC0DF00FC0F6FF8D
:1052000010C0F7FF85EC0DF0FA0E9DEC0BF0B4EC3E
:1052100029F0D8A412EF29F0110E0F26D8B0102AC9
:1052200019EF29F0D8A026EF29F0130E0F26D8B0D9
:10523000102A0FC0F6FF10C0F7FFF86A0900F5CF7B
:105240000FF00900F5CF10F0FBEF28F025EC25F06A
:1052500081EC1EF0D8A0FBEF28F0150E0F26D8B079
:10526000102A0FC0F6FF10C0F7FFF86A0900F5CF4B
:105270000AF00900F550CEC0E1FFCFC0E2FF0AC03E
:10528000E7FF12000F0BE8B6080B0C0DF3CF13F07D
:10529000F4CF14F00001380E1326710E1422CC0E38
:1052A0000FEC0DF013C0F6FF14C0F7FF85EC0DF006
:1052B000FA0E9DEC0BF0B4EC29F0D8A466EF29F0BF
:1052C000050E1326D8B0142A6DEF29F0D8A07AEF76
:1052D00029F0070E1326D8B0142A13C0F6FF14C005
:1052E000F7FFF86A0900F5CF13F00900F5CF14F0C5
:1052F0004FEF29F025EC25F081EC1EF0D8A04FEF00
:1053000029F0090E1326D8B0142A13C0F6FF14C0D2
:10531000F7FFF86A0900F5CFE8FF1200040E93ECDE
:1053200008F0040E93EC08F0C5C0E8FFC35EC6C0E9
:10533000E8FFC45AC4BEA7EF29F0640EC35E000E96
:10534000C45AC4BEB1EF29F0D884D8901200640EBC
:10535000C326000EC422C4AEB1EF29F0D894D88081
:105360001200D894D8901200050E93EC08F0050EA8
:1053700093EC08F0C7C0E8FFC35EC8C0E8FFC45A9A
:10538000C4BED1EF29F0640EC35E000EC45AC4BE81
:10539000E1EF29F0C466C368C3CFF0F0D884D89099
:1053A0001200640EC326000EC422C4AEE1EF29F041
:1053B000C31EC41EC466C368C3CFF0F0D894D8809F
:1053C0001200D894D8901200DEEF2AF0800E0FEC75
:1053D0000DF0000EF86E670EF76E680EF66E85EC37
:1053E0000DF02BEF2BF00101800E1E6F670E1F6F6B
:1053F00001016C0E206F690E216F6EEC2AF0A7EC94
:105400001EF000C2E8FF38EC1FF065EC1FF0120040
:105410000101980E1E6F670E1F6F01015E0E206F57
:105420006A0E216F6EEC2AF0FFEF29F00101B00E39
:105430001E6F670E1F6F0101480E206F6C0E216FEB
:105440006EEC2AF0FFEF29F00101C80E1E6F670E07
:105450001F6F0101A40E206F710E216F6EEC2AF0F8
:10546000FFEF29F00101E00E1E6F670E1F6F0101B3
:10547000720E206F780E216F6EEC2AF0FFEF29F08C
:105480000001DD6B0101F80E1E6F670E1F6F010139
:105490007C0E206F7E0E216F6EEC2AF0FFEF29F05C
:1054A0000101100E1E6F680E1F6F0101C40E206FE8
:1054B000820E216F6EEC2AF0FFEF29F00101280E19
:1054C0001E6F680E1F6F01013E0E206F860E216F4A
:1054D0006EEC2AF0FFEF29F003EF32F04EEC25F0EE
:1054E00020C10DF021C10EF087EC25F00DC020F198
:1054F0000EC021F1EAC026F1EBC027F100011150E6
:10550000090AD8A4D0EF2AF00FC00DF010C00EF099
:1055100087EC25F00DC022F10EC023F1EAC028F17E
:10552000EBC029F100011150090AD8A4B8EF2AF004
:105530000FC00DF010C00EF087EC25F00DC024F167
:105540000EC025F1EAC02AF1EBC02BF15EEC26F08B
:105550000001CDB1BEEF2AF02AC10FF02BC110F02F
:1055600052EC26F024C10DF025C10EF09CEF2AF07C
:105570005EEC26F00001CDB1D5EF2AF028C10FF086
:1055800029C110F052EC26F020C10DF021C10EF01F
:1055900064EC0DF022C10DF023C10EF088EF2AF06B
:1055A0005EEC26F00001CDB1120026C10FF027C13C
:1055B00010F052EC26F06EEF2AF0120000C2E8FF65
:1055C000B8EC1EF0800E0FEC0DF0000EF86E650EBC
:1055D000F76E6A0EF66E85EC0DF08D0E0FEC0DF089
:1055E000020100510001136E146A156A166AE3EC99
:1055F0000DF0CDEC05F0FA0E9DEC0BF0B4EC29F0BB
:10560000D8A40DEF2BF0610E0201002B0063DEEF3A
:105610002AF0010E006FDEEF2AF0D8A01BEF2BF06E
:1056200002010007000E0063DEEF2AF0600E0201A7
:10563000006FDEEF2AF081EC1EF0D8A0FEEF2AF01A
:1056400000C2E8FF0DEC1FF000C2E8FFE8CFA5F0B4
:10565000A7EC1EF01200C00E0FEC0DF0CDEC05F023
:10566000000EE16E030EE26E960E9DEC0BF0C00E86
:10567000E1240FEC0DF0E75000EC0DF0C00EE1243A
:105680000FEC0DF00E0E0FEC0DF08EEC29F0D8A4FF
:1056900053EF2BF0E12A0F0EE16434EF2BF0000EF4
:1056A000E16E34EF2BF0D8A05FEF2BF0E106FF0E98
:1056B000E16234EF2BF00F0EE16E34EF2BF0B4EC1F
:1056C00029F0D8A46AEF2BF0E72A7A0EE760E76E9C
:1056D00034EF2BF0D8A073EF2BF0E706200EE76431
:1056E000E76E34EF2BF081EC1EF0D8A045EF2BF0E5
:1056F0000C0E0FEC0DF000C2E8FF38EC1FF01200AA
:105700000DC02CF10EC02DF10FC02EF110C02FF1E5
:10571000D0C00DF0D1C00EF00001E80E0F6E030EE8
:10572000106E67EC10F00001000E176E010E186E7F
:105730006BEC11F013C0D0F014C0D1F00001D251C5
:10574000D027D351D123D4C00DF0D5C00EF0000125
:10575000E80E0F6E030E106E67EC10F00001000EE5
:10576000176E010E186E6BEC11F0D2C0D4F0D3C0DE
:10577000D5F01350D45F1450D55BD0C00DF0D1C01C
:105780000EF062EC1EF00DC0D0F00EC0D1F0D2C011
:105790000DF0D3C00EF062EC1EF00DC0D2F00EC0C2
:1057A000D3F0D4C00DF0D5C00EF062EC1EF00DC0E9
:1057B000D4F00EC0D5F02CC10DF02DC10EF02EC1CD
:1057C0000FF02FC110F012000DC02CF10EC02DF102
:1057D0000FC02EF110C02FF1D0C00DF0D1C00EF0CF
:1057E0000001E80E0F6E030E106E67EC10F0000162
:1057F000000E176E010E186E6BEC11F0D2C0D0F0D7
:10580000D3C0D1F000011350D0271450D12313502E
:10581000D25F1450D35BD0C00DF0D1C00EF062EC5B
:105820001EF00DC0D0F00EC0D1F0D2C00DF0D3C02C
:105830000EF062EC1EF00DC0D2F00EC0D3F02CC101
:105840000DF02DC10EF02EC10FF02FC110F012007F
:105850000DC02CF10EC02DF10FC02EF110C02FF194
:10586000D0C00DF0D1C00EF0D2510D5ED3510E5A02
:105870000001000E0F6E010E106E67EC10F00001BB
:10588000E80E176E030E186E6BEC11F013C0D0F01B
:1058900014C0D1F0D2C00DF0D3C00EF0D4510D5EC3
:1058A000D5510E5A0001000E0F6E010E106E67ECFE
:1058B00010F00001E80E176E030E186E6BEC11F07D
:1058C00013C0D4F014C0D5F02CC10DF02DC10EF0D2
:1058D0002EC10FF02FC110F012000DC02CF10EC020
:1058E0002DF10FC02EF110C02FF1D0C00DF0D1C09E
:1058F0000EF00001D2510D5ED3510E5A0001000E80
:105900000F6E010E106E67EC10F00001D00E176ED6
:10591000070E186E6BEC11F013C0D0F014C0D1F06C
:10592000D0C00DF0D1C00EF00001E80E0F6E030ED6
:10593000106E67EC10F00001000E176E010E186E6D
:105940006BEC11F000011350D2271450D3232CC15B
:105950000DF02DC10EF02EC10FF02FC110F012006E
:105960000DC02CF10EC02DF10FC02EF110C02FF183
:105970000001BEA1E8EF2CF0000E00010F18D8B412
:10598000D3EF2CF0D2C013F0D3C014F0D89013365C
:105990001436D051135ED151145A13C0D4F014C030
:1059A000D5F0E8EF2CF0000E00010F18D8B4E8EFA6
:1059B0002CF0D2C013F0D3C014F0D89013361436A4
:1059C000D451135ED551145A13C0D0F014C0D1F085
:1059D0002CC10DF02DC10EF02EC10FF02FC110F013
:1059E00012003C0E0001B86F0001110EB56F030EDE
:1059F000B66F0001D00EB36F000EB46F0B0EB76F11
:105A000056EC23F0DB6B80EC2BF012003A0E000119
:105A1000B86F00011C0EB56F030EB66FF9EF2CF0D6
:105A20003E0E0001B86F0001270EB56F030EB66F72
:105A3000F9EF2CF00001110EB36F030EB46FB0EC50
:105A40002CF0DBA1D86B28EC2CF00001D00EB56F48
:105A5000000EB66F0B0EB76F56EC23F00001B86B5B
:105A6000120000011C0EB36F030EB46F1FEF2DF078
:105A70000001270EB36F030EB46F1FEF2DF00DC0A2
:105A80002CF10EC02DF10FC02EF110C02FF103012B
:105A900032C30DF033C30EF00001E80E0F6E030E9B
:105AA000106E67EC10F00001000E176E010E186EFC
:105AB0006BEC11F013C032F314C033F30301345113
:105AC0003227355133232CC10DF02DC10EF02EC1DC
:105AD0000FF02FC110F012000DC02CF10EC02DF1EF
:105AE0000FC02EF110C02FF132C30DF033C30EF0F2
:105AF0000301345100010D5E0301355100010E5ABE
:105B00000001000E0F6E010E106E67EC10F0000128
:105B1000E80E176E030E186E6BEC11F013C032F323
:105B200014C033F32CC10DF02DC10EF02EC10FF0B7
:105B30002FC110F00001B86B1200420E0001B86FC7
:105B400000013A0EB56F030EB66F0001D00EB36FB1
:105B5000000EB46F040EB76F56EC23F0E4EC2BF09C
:105B60001200440E0001B86F00013E0EB56F030E27
:105B7000B66FA5EF2DF0460E0001B86F0001420E82
:105B8000B56F030EB66FA5EF2DF000013A0EB36F9F
:105B9000030EB46F6DEC2CF00001D00EB56F000E4B
:105BA000B66F040EB76F56EC23F00001B86B12000D
:105BB00000013E0EB36F030EB46FCAEF2DF000016B
:105BC000420EB36F030EB46FCAEF2DF00001460E04
:105BD000B56F030EB66F0001D00EB36F000EB46F39
:105BE000060EB76F56EC23F080EC2BF0120028EC79
:105BF0002CF00001D00EB56F000EB66F0001460EFE
:105C0000B36F030EB46F060EB76F56EC23F00001AE
:105C1000B86B1200AEC2B9F0AFC2BAF0B0C2BBF0FE
:105C2000B1C2BCF01200CEC0B5F0CFC0B6F00001DA
:105C3000DC0EB36F000EB46F050EB76F56EC23F099
:105C4000CEC0B3F0CFC0B4F00001DC51E83A0F0B86
:105C5000E46FE36BDDBFE31FE16BDF51DDBDE16F9F
:105C6000E26BE051DDBBE26F0F0EE117E217DD17CB
:105C7000DC1712000001E451E83AF00BDC13E3BF3B
:105C8000DD8FE151E812D8B449EF2EF0E151DF6F1A
:105C9000DD8DE251E812D8B451EF2EF0E251E06F01
:105CA000DD8B0001DC0EB56F000EB66F050EB76F11
:105CB00056EC23F0120010C4DFF011C4E0F0120023
:105CC000DFC010F4E0C011F4120012C4DFF013C4FE
:105CD000E0F01200DFC012F4E0C013F4120014C4AC
:105CE000DFF015C4E0F01200DFC014F4E0C015F4DA
:105CF00012000001DBAF12000301196B246B2F6B44
:105D000012000001DBAF1200A7C313F0A8C314F008
:105D1000835113268451142213C0A7F314C0A8F38F
:105D2000A9C313F0AAC314F0855113268651142277
:105D300013C0A9F314C0AAF3ABC313F0ACC314F09F
:105D4000875113268851142213C0ABF314C0ACF34F
:105D500012000001DBAF12000301A76BA86BA96B57
:105D6000AA6BAB6BAC6B12000001B96BB92B600E68
:105D70000001BB6F12000001DD51DD67C1EF2EF0A5
:105D80001200020100C20AF0006F00010AC0DDF03B
:105D900038EC1FF00001DDC00AF002010AC000F279
:105DA00012000001DBAF120003011951196B18C377
:105DB0000AF000010D6E0E6AE8BE0E680D360E3652
:105DC0000001640E0F6E000E106E67EC10F00AC03A
:105DD00017F0186A6BEC11F013500301A7270001AC
:105DE00014500301A82303012451246B23C30AF098
:105DF00000010D6E0E6AE8BE0E680D360E3600010B
:105E0000640E0F6E000E106E67EC10F00AC017F0F3
:105E1000186A6BEC11F013500301A927000114500C
:105E20000301AA2303012F512F6B2EC30AF0000197
:105E30000D6E0E6AE8BE0E680D360E360001640E59
:105E40000F6E000E106E67EC10F00AC017F0186AA3
:105E50006BEC11F013500301AB2700011450030148
:105E6000AC2312000001DBAF120064EC32F0120030
:105E700056EC23F012000001D00EB36F000EB46F89
:105E8000CEC0B5F0CFC0B6F00B0EB76F56EC23F016
:105E90000001D00EB56F000EB66FCEC0B3F0CFC00C
:105EA000B4F00B0EB76F12000201D890A2371200A7
:105EB0000201D890A23312000001E9AF120011ECE8
:105EC00010F0120013C20FF014C210F0030E000104
:105ED000A06F13EC31F00FC013F210C014F21200D7
:105EE000A9C20FF0AAC210F00D0E0001A06F13ECB2
:105EF00031F00FC0A9F210C0AAF212000001DBAF0E
:105F000012000501006B016B0201B8691200C9ECB7
:105F10000BF012000001CE51B36F020EB46FCF51DF
:105F200000011F6E030E7EEC08F014C08BF015C04C
:105F30008CF0C00E0FEC0DF0000EF86E8C0EF76EAC
:105F4000560EF66E85EC0DF081EC1EF0D8A0A4EF95
:105F50002FF000011F507EEC08F014C06DF015C04A
:105F60006EF014C06FF015C070F0FA0E9DEC0BF0DF
:105F7000C00E0FEC0DF0000EF86E8C0EF76E680E72
:105F8000F66E85EC0DF081EC1EF0D8A0C3EF2FF07B
:105F900000011F507EEC08F014C06BF015C06CF0CF
:105FA000FA0E9DEC0BF000016B516D276C516E23C6
:105FB0006E336D336E9F6FC017F070C018F0000124
:105FC000E80E146E030E156E136A166A6B51175E97
:105FD0006C51185A18321732187E196A1A6A6BEC0B
:105FE00011F013C06BF014C06CF000016B0EB56FB4
:105FF000000EB66F040E0001B76F56EC23F01200CE
:106000000001CE51B36F020EB46FCF5100011F6E6D
:10601000C00E0FEC0DF0000EF86E8C0EF76E560EE3
:10602000F66E85EC0DF081EC1EF0D8A013EF30F089
:1060300000011F507EEC08F014C06BF015C06CF02E
:10604000FA0E9DEC0BF0C00E0FEC0DF0000EF86E8A
:106050008C0EF76E680EF66E85EC0DF081EC1EF07E
:10606000D8A02EEF30F000011F507EEC08F014C0D5
:106070006DF015C06EF0FA0E9DEC0BF00001E80E0D
:10608000146E030E156E136A166A6BC017F06CC09F
:1060900018F0196A1A6A00016D51175E6E51185A8C
:1060A00018AE54EF30F0FF0E196E1A6E6BEC11F053
:1060B00013C06BF014C06CF000016B0EB56F000ED6
:1060C000B66F040E0001B76F56EC23F0120000010A
:1060D000CE51B36F020EB46FCF5100011F6EC00ED0
:1060E0000FEC0DF0000EF86E8C0EF76E440EF66E8F
:1060F00085EC0DF081EC1EF0D8A07AEF30F00001B5
:106100001F507EEC08F0000113361436153614C00B
:106110006DF015C06EF0FA0E9DEC0BF0C00E0FEC9A
:106120000DF0000EF86E8C0EF76E560EF66E85ECC6
:106130000DF081EC1EF0D8A099EF30F000011F5057
:106140007EEC08F0000113361436153614C06BF0DF
:1061500015C06CF0FA0E9DEC0BF0C00E0FEC0DF0BC
:10616000000EF86E8C0EF76E680EF66E85EC0DF074
:1061700081EC1EF0D8A0B8EF30F000011F507EEC8B
:1061800008F0000113361436153614C06FF015C030
:1061900070F0FA0E9DEC0BF00001E80E146E030E89
:1061A000156E136A166A6BC017F06CC018F0196A86
:1061B0001A6A00016D51175E6E51185A18AEE2EF5F
:1061C00030F0FF0E196E1A6E6BEC11F013C06BF00D
:1061D00014C06CF00001E80E146E030E156E136A05
:1061E000166A6DC017F06EC018F0196A1A6A0001BD
:1061F0006F51175E7051185A18AE00EF31F0FF0E54
:10620000196E1A6E6BEC11F013C06FF014C070F0C1
:1062100000016B0EB56F000EB66F060E0001B76F72
:1062200056EC23F01200140E9DEC0BF00001A0516F
:1062300093EC08F0C00E0FEC0DF0000EF86E690E36
:10624000F76E000EF66E85EC0DF0CB0E0FEC0DF038
:1062500069C00DF06AC00EF067EC10F01450136EB8
:106260001550146E156A15EC0EF0200E0A6E300EE5
:1062700025640AC025F0255000EC0DF0265000ECF6
:106280000DF02E0E00EC0DF0275000EC0DF0285014
:1062900000EC0DF0B4EC29F0D8A455EF31F000017A
:1062A0000F2AD8B4102A13EF31F0D8A05FEF31F0E5
:1062B00000010F06FF0E0F60100613EF31F081ECA6
:1062C0001EF0D8A013EF31F012000201FF0EA563FB
:1062D00077EF31F000019D510FEC0DF0000EF86EDC
:1062E000650EF76E8E0EF66E85EC0DF01200020153
:1062F000D1B195EF31F0D1A395EF31F000019D516F
:106300000FEC0DF0000EF86E650EF76E7C0EF66E5B
:1063100085EC0DF000019D51080F0FEC0DF002010E
:10632000310EA52500EC0DF012000201D1A1CAEF3B
:1063300031F0D1B3CAEF31F000019D510FEC0DF0F7
:10634000000EF86E650EF76EE80EF66E85EC0DF039
:1063500000019D510E0F0FEC0DF00201300EA5252E
:1063600000EC0DF00201A551D890E836500F000165
:10637000136E146A156A166A15EC0EF000019D5131
:10638000040F0FEC0DF0285000EC0DF0295000EC3C
:106390000DF012000201D1A11200D1A312000001E0
:1063A0009D510FEC0DF0000EF86E660EF76E540E58
:1063B000F66E85EC0DF000019D510D0F0FEC0DF008
:1063C0000201A55101010E250001136E146A156A20
:1063D000166AE3EC0DF00201A551D890E836010FE2
:1063E0000001136E146A156A166A15EC0EF00001AE
:1063F0009D51040F0FEC0DF0285000EC0DF02950CA
:1064000000EC0DF012000301FF0EAD6318EF32F047
:10641000C00E0FEC0DF0000EF86E650EF76E8E0ECE
:10642000F66E85EC0DF0FA0E9DEC0BF024EF32F0D9
:106430000301AD510201A56FC00E00019D6F65EC17
:1064400031F0FA0E9DEC0BF0B4EC29F0D8A434EF47
:1064500032F0010110510301AD2BAD6303EF32F0B7
:10646000FF0EAD6F03EF32F0D8A044EF32F003011E
:10647000AD07FE0EAD6303EF32F001011051E806E7
:106480000301AD6F03EF32F081EC1EF0D8A024EFD2
:1064900032F000C2E8FF38EC1FF01200000EF86E78
:1064A0008C0EF76E7A0EF66E000E0A6E020EE26E1B
:1064B000000EE16E0900F550E66E0A060900F5507F
:1064C000E66E0A2E5AEF32F0000EF86E8D0EF76E61
:1064D0007A0EF66E000E0A6E030EE26E000EE16E8C
:1064E0000900F550E66E0A060900F550E66E0A2E20
:1064F00070EF32F0000EF86E8E0EF76E7A0EF66EBA
:10650000000E0A6E040EE26E000EE16E0900F550F8
:10651000E66E0A060900F550E66E0A2E86EF32F0A6
:106520001200202020202020202020202020202099
:1065300020200000204D6963726F53746172203215
:10654000303030200000202056657273696F6E2055
:10655000322E30652020000041444320434820581B
:1065600058203D205858585800002020204169727A
:1065700063726166742023202020000020202020E8
:106580002035332E58204D487A202020000020202E
:1065900020202020204F46462020202020200000C0
:1065A000204163636570743F20596573204E6F20EE
:1065B00000002050726573732020204F7074696F43
:1065C0006E200000202020202020200020202020DD
:1065D00053747564656E74202020202000002059BB
:1065E0006573204E6F2000002035302E5858204D06
:1065F000487A202043485820000078426C6420529A
:10660000504D203D2078787878780000526574727B
:106610006163747320617265205550210000202051
:10662000466F726D617420466C61736820200000B3
:106630002020466F726D6174696E672E2E2E2020A9
:106640000000202020436F7079696E672E2E2E2067
:10665000202000002037322E5858204D487A204301
:1066600048585820000052454320566F6C74733DC3
:106670002058582E585800005468726F74746C6516
:10668000202041646A7573740000202041494C2029
:10669000442F5220484947482020000020204149EB
:1066A0004C20442F5220204C4F5720200000202007
:1066B000454C4520442F522048494748202000009F
:1066C0002020454C4520442F5220204C4F5720205D
:1066D0000000202052554420442F5220484947486A
:1066E00020200000202052554420442F5220204CCE
:1066F0004F5720200000202020534E415020524967
:106700004748542020200000202020534E41502094
:10671000204C454654202020000020202041555484
:106720004F20205452494D202020000020202020BE
:106730002050524553455420202020200000202086
:106740002043414C49425241544520202020000022
:1067500053656C656374202041697263726166746D
:1067600000686758680000002041697263726166C2
:106770007420206E616D6520008067506704000002
:1067800020202020202054696D65722020202020A8
:106790000098676867080000202020202020536EA2
:1067A000617020202020202000B06780670C00004E
:1067B0002020202020536572766F73202020202017
:1067C00000C867986710000020202020204D6978BD
:1067D000657273202020202000E067B0671400005D
:1067E00020202020205377697463682020202020F7
:1067F00000F867C867180000202020204F707469D7
:106800006F6E732020202020001068E0671C0000BD
:1068100020536861726564204F7074696F6E7320D5
:10682000002868F867200000202053797374656D94
:1068300020536574757020200040681068240000A3
:1068400053656C656374204672657175656E637916
:106850000058682868280000202020202020455863
:10686000495420202020202000506740682C000040
:10687000456E61626C652020202020202020202091
:1068800000005265736574203F20202020202020C6
:10689000202000005A65726F20203F2020202020F9
:1068A000202020200000436C656172203F202020C2
:1068B00020202020202000004169726372616674EC
:1068C00020232020202020200000546F2041465407
:1068D000202320202020202020200000426C616402
:1068E0006573203D202020202020202000004678B5
:1068F0006420467273742020202020202020000075
:10690000566F6C747320202020202020202020200F
:106910000000576964746820202020202020202057
:10692000202000004368616E6E656C73202020207B
:106930002020202000004E656753686966743F2060
:106940002020202020200000506F73203D20202098
:10695000202020202020202000004761696E202078
:106960002020202020202020202000002020202067
:1069700020204D6F6465202020202020008869FCA5
:10698000690080166ABD03004D696E7574657320D9
:10699000202020202020202000A8696C690540BF0D
:1069A0000300000000FF00005365636F6E647320F6
:1069B000202020202020202000C86988690540BEB2
:1069C0000300000000FF000020456E61626C65203E
:1069D000205377697463682000E269A8690680C063
:1069E00003005468726F74746C652020202020208E
:1069F000202000FC69C8690100C1030045584954C2
:106A0000202020202020202020202020006C69E24F
:106A1000690300CD00002020202055502054696DCE
:106A2000657220202020002E6A466A000000202087
:106A300020446F776E2054696D65722020200046D7
:106A40006A166A010000446F776E202053746F70DD
:106A50002054696D657200166A2E6A020000535256
:106A60002041494C20202020202020202020007E72
:106A70006A2E6C01404C030000FF007E0000535260
:106A800020454C4520202020202020202020009E32
:106A90006A5E6A01404E030000FF007E0000535210
:106AA000205255442020202020202020202000BEDD
:106AB0006A7E6A014050030000FF007E00005352CE
:106AC000205448542020202020202020202000DE98
:106AD0006A9E6A014052030000FF007E000053528C
:106AE0002041494C203F202020202020202000F859
:106AF0006ABE6A03004D0300535220454C45203FB7
:106B0000202020202020202000126BDE6A03004F6E
:106B10000300535220525544203F202020202020A3
:106B20002020002C6BF86A030051030053522054BC
:106B30004854203F202020202020202000466B1297
:106B40006B0300530300534C2041494C202020206C
:106B500020202020202000666B2C6B014054030075
:106B600000FF007E0000534C20454C452020202093
:106B700020202020202000866B466B014056030019
:106B800000FF007E0000534C20525544202020205E
:106B900020202020202000A66B666B0140580300B7
:106BA00000FF007E0000534C205448542020202039
:106BB00020202020202000C66B866B01405A030055
:106BC00000FF007E0000534C2041494C203F202014
:106BD00020202020202000E06BA66B03005503003E
:106BE000534C20454C45203F2020202020202020B1
:106BF00000FA6BC66B0300570300534C20525544F8
:106C0000203F202020202020202000146CE06B0357
:106C100000590300534C20544854203F202020208A
:106C200020202020002E6CFA6B03005B03004558E7
:106C30004954202020202020202020202020005ED9
:106C40006A146C0300CD00002020202041696C658F
:106C5000726F6E202020202000686C626D09867C97
:106C60006D0000345AE2590020202020456C6576E2
:106C700061746F722020202000886C486C09867C2B
:106C80006D0000625A0C5A002020202020527564AA
:106C9000646572202020202000A86C686C09867C26
:106CA0006D0000705A205A00202020205468726F16
:106CB00074746C652020202000C86C886C09867272
:106CC0006E0000D85A7E5A00202020202020434801
:106CD000352020202020202000E86CA86C09866444
:106CE0006F00008A5B3A5B00202020202020434870
:106CF000362020202020202000086DC86C098664E2
:106D00006F0000B05B625B00202020202020434801
:106D1000372020202020202000286DE86C09866480
:106D20006F0000BE5B765B002020202020204348BF
:106D3000382020202020202000486D086D0986BAC8
:106D40006F0000EE5BCC5B0020202020537562209A
:106D50005472696D7320202000626D286D09802EA9
:106D60007000455849542020202020202020202039
:106D7000202000486C486D0300CD000052542F4481
:106D8000574E20202020202020202020009A6D58BF
:106D90006E0202D0000000145C0043656E746572E0
:106DA0002020202020202020202000B86D7C6D0293
:106DB00002D2000000145C004C542F5550202020BB
:106DC000202020202020202000D66D9A6D0202D4A1
:106DD000000000145C004475616C205261746520F1
:106DE00020202020202000F06DB86D0100D600008A
:106DF0005472696D20202020202020202020202077
:106E0000000A6ED66D0100D7000041542052535441
:106E10002020202020202020202000246EF06D0340
:106E200000DB00004578706F20484920202020209A
:106E300020202020003E6E0A6E0100D90000457817
:106E4000706F204C4F5720202020202020200058F9
:106E50006E246E0100DA000045584954202020209D
:106E60002020202020202020007C6D3E6E0300CDBD
:106E70000000486967682020202020202020202052
:106E8000202000906E026F020332034000145C0069
:106E90004C6F772020202020202020202020202020
:106EA00000AE6E726E020334034000145C00547234
:106EB000696D20202020202020202020202000C8B4
:106EC0006E906E01003603005472696D204D6F6440
:106ED000652020202020202000E46EAE6E00001CE3
:106EE0006F370300507265736574202020202020C6
:106EF0002020202000026FC86E02033803400014D7
:106F00005C004558495420202020202020202020AB
:106F1000202000726EE46E0300CD00005472696D93
:106F2000204D6F6465204E4F524D414C00346F4CE4
:106F30006F0000005472696D204D6F646520202041
:106F4000204C4F57004C6F1C6F0100005472696D4C
:106F5000204D6F646520202048494748001C6F344D
:106F60006F020000486967682F557020202020209C
:106F70002020202000826FA06F0202D000000014A9
:106F80005C004C6F772F44574E202020202020207B
:106F9000202000A06F646F0202D2000000145C0089
:106FA0004558495420202020202020202020202027
:106FB00000646F826F0300CD00004120202020205C
:106FC0002020202020202020202000D86F147002B4
:106FD00003D0004800145C00422020202020202004
:106FE000202020202020202000F66FBA6F0203D23C
:106FF000004800145C004320202020202020202076
:10700000202020202020001470D86F0203D40048D4
:1070100000145C00455849542020202020202020C6
:107020002020202000BA6FF66F0300CD00004169D8
:107030006C65726F6E202020202020202020004CC4
:10704000701E71010208040000084B00456C657653
:1070500061746F722020202020202020006A702E72
:1070600070010209040000084B00527564646572E7
:10707000202020202020202020200088704C70011B
:10708000020A040000084B005468726F74746C6547
:10709000202020202020202000A6706A7001020BF2
:1070A000040000084B0043483520202020202020E9
:1070B00020202020202000C470887001020C0400D1
:1070C00000084B004348362020202020202020208C
:1070D0002020202000E270A67001020D04000008AC
:1070E0004B00434837202020202020202020202033
:1070F0002020000071C47001020E040000084B0043
:10710000434838202020202020202020202020201C
:10711000001E71E27001020F040000084B00457868
:107120006974202020202020202020202020002ED4
:107130007000710300CD00004E6F6E6500447198C1
:10714000710000002041494C00507138710100006D
:1071500020454C45005C71447102000020525544AA
:107160000068715071030000205448540074715C31
:1071700071040000204348350080716871050000EB
:1071800020434836008C7174710600002043483754
:107190000098718071070000204348380038718CD6
:1071A00071080000202020204D49584552203141CF
:1071B0002020202000C4715C740986C4745C0374B0
:1071C0005C265C00202020204D4958455220314249
:1071D0002020202000E471A4710986C47461037426
:1071E0005C265C00202020204D4958455220314328
:1071F00020202020000472C4710986C474660374C0
:107200005C265C00202020204D4958455220314406
:1072100020202020002472E4710986C4746B03745A
:107220005C265C00202020204D49584552203241E8
:107230002020202000447204720986C474700374F4
:107240005C265C00202020204D49584552203242C7
:107250002020202000647224720986C4747503748F
:107260005C265C00202020204D49584552203243A6
:107270002020202000847244720986C4747A03742A
:107280005C265C00202020204D4958455220324485
:107290002020202000A47264720986C4747F0374C5
:1072A0005C265C00202020204D4958455220334167
:1072B0002020202000C47284720986C47484037460
:1072C0005C265C00202020204D4958455220334246
:1072D0002020202000E472A4720986C474890374FB
:1072E0005C265C00202020204D4958455220334325
:1072F00020202020000473C4720986C4748E037495
:107300005C265C00202020204D4958455220334403
:1073100020202020002473E4720986C4749303742F
:107320005C265C0020202041494C20746F2052557F
:10733000442020200044730473098676749303C0AC
:107340005CB65C0020202052554420746F204149D7
:107350004C2020200064732473098676749303D430
:107360005CCA5C0020202052554420746F20454C9C
:10737000452020200084734473098676749303E8C3
:107380005CDE5C0020202054485420746F20454C63
:107390004520202000A0736473018816045A6900F8
:1073A0002020202020565441494C202020202020FD
:1073B00000BC738473038898037068002020202029
:1073C00020454C45564F4E202020202000D873A049
:1073D0007303889903706800202020204455414C95
:1073E0002041494C2020202000F273BC730980CA40
:1073F0007500202020204455414C20454C4520203C
:107400002020000C74D8730980667600202020208C
:1074100054485420484F4C4420202020002674F229
:10742000730980B476002020202049444C45202058
:107430005550202020200040740C740980027700F1
:1074400020204D6978657220206F7264657220205B
:10745000005C7426740388A403EE68004558495400
:1074600020202020202020202020202000A4714047
:10747000740300CD0000506F73206761696E202097
:10748000202020202020009074AA740100DF00003A
:107490004E6567206761696E202020202020202013
:1074A00000AA7476740100E0000045584954202079
:1074B000202020202020202020200076749074039B
:1074C00000CD000046726F6D20202020202020205B
:1074D0002020202000DE74B0750400DC0000546120
:1074E000626C65202020202020202020202000FA0F
:1074F00074C47400006A77E40000546F20202020D8
:1075000020202020202020202020001475DE74045C
:1075100000DD00005265706C616365202020202032
:1075200020202020002E75FA740300E300005A503A
:107530002020202020202020202020202020004843
:107540007514750100DE0000506F73206761696E6D
:1075500020202020202020200062752E750100DFD1
:107560000000506F7320496E6420202020202020CE
:107570002020007C7548750400E100004E656720FE
:107580006761696E202020202020202000967562EF
:10759000750100E000004E656720496E64202020E0
:1075A00020202020202000B0757C750400E200001F
:1075B0004558495420202020202020202020202011
:1075C00000C47496750300CD0000456E61626C6561
:1075D0002020202020202020202000E4754C76034D
:1075E000009A03005265762043483720202020204F
:1075F0002020202000FE75CA7503009B030044492B
:107600004646202020202020202020202020001856
:1076100076E47501009C0300466C617020202020F8
:107620002020202020202020003276FE7501009DA1
:10763000030043524F5720202020202020202020CC
:107640002020004C7618760300C6030045584954A4
:1076500020202020202020202020202000CA753239
:10766000760300CD0000456E61626C65202020200D
:107670002020202020200080769A76030017040026
:1076800052657620434836202020202020202020CC
:10769000009A766676030018040045584954202065
:1076A00020202020202020202020006676807603C5
:1076B00000CD0000456E61626C65202020202020F6
:1076C0002020202000CE76E87603009E0300506F35
:1076D000736974696F6E202020202020202000E82C
:1076E00076B47601009F030045584954202020209D
:1076F000202020202020202000B476CE760300CD4C
:107700000000456E61626C65202020202020202032
:107710002020001C7750770300A00300506F73698E
:1077200074696F6E204120202020202000367702CF
:10773000770100A10300506F736974696F6E204276
:107740002020202020200050771C770100A2030079
:10775000455849542020202020202020202020206F
:1077600000027736770300CD00005461626C65201B
:107770002020202020204E6F6E650082775A7800EE
:1077800000004169726372616674205461626C65C5
:107790002031009A776A770900004169726372614B
:1077A0006674205461626C65203200B27782770A79
:1077B0000000476C6F6162616C205461626C6520EF
:1077C000203100CA779A77010000476C6F616261CF
:1077D0006C205461626C6520203200E277B277023F
:1077E0000000476C6F6162616C205461626C6520BF
:1077F000203300FA77CA77030000476C6F6162613B
:107800006C205461626C65202034001278E27704A9
:107810000000476C6F6162616C205461626C65208E
:107820002035002A78FA77050000476C6F616261A5
:107830006C205461626C6520203600427812780614
:107840000000476C6F6162616C205461626C65205E
:107850002037005A782A78070000476C6F61626110
:107860006C205461626C65202038006A7742780889
:107870000000202020202041494C2044522020207C
:107880002020008C78607A0680AE03002020202023
:1078900020454C45204452202020202000A678720C
:1078A000780680AF03002020202020525544204439
:1078B00052202020202000C0788C780680B0030061
:1078C00020202020205052455345542020202020A5
:1078D00000DA78A6780680B10300202020204D49E8
:1078E0005845522020312020202000F478C078060E
:1078F00080B20300202020204D49584552202032DC
:1079000020202020000E79DA780680B303002020A2
:1079100020204D4958455220203320202020002887
:1079200079F4780680B403002020202020204348EA
:1079300035202020202020200042790E790680B5B5
:107940000300202020204155544F205452494D20FF
:107950002020005C7928790680B6030020202020B2
:1079600020434838204120202020202000767942E2
:10797000790680B703002020202020434838204289
:107980002020202020200090795C790680B8030018
:107990002020202020434838204320202020202061
:1079A00000AA7976790680B9030020202020534E62
:1079B0004150202052202020202000C479907906B8
:1079C00080BB030020202020534E415020204C201B
:1079D0002020202000DE79AA790680BC03002054F4
:1079E00068726F74746C652020486F6C642000F8B6
:1079F00079C4790680C2030020202049646C652088
:107A0000557020203120202000127ADE790680C3B4
:107A1000030020202049646C65205570202032200E
:107A20002020002C7AF8790680C403002020202032
:107A3000202043524F5720202020202000467A1239
:107A40007A0680C50300205472696767657220500A
:107A50006F696E74732000607A2C7A09807A7A00DC
:107A6000455849542020202020202020202020205C
:107A7000007278467A0300CD000041696C65726F30
:107A80006E205472696720506F7300967AEA7A010B
:107A900088C903486900456C657661746F7220542B
:107AA000726720506F7300B27A7A7A0188CA0348ED
:107AB00069005275646465722020547269672050B1
:107AC0006F7300CE7A967A0188CB034869005468B8
:107AD000726F74746C652054726720506F7300EA83
:107AE0007AB27A0188CC034869004558495420206D
:107AF00020202020202020202020007A7ACE7A0307
:107B000000CD0000202020202020204F4E202020CB
:107B100020202020001C7B647E10000020202020DC
:107B20002020204F464620202020202000347B04A7
:107B30007B2000005357412020202020202020209F
:107B400020204F4E004C7B1C7B00000053574120EF
:107B50002020202020202020204F464600647B3417
:107B60007B8000005357422020202020202020200E
:107B700020204F4E007C7B4C7B010000535742205D
:107B80002020202020202020204F464600947B6487
:107B90007B810000535743202020202020202020DC
:107BA00020204F4E00AC7B7C7B02000053574320CB
:107BB0002020202020202020204F464600C47B94F7
:107BC0007B8200005357442020202020202020507A
:107BD0005245535300DC7BAC7B8300005357442059
:107BE000202020202052454C4541534500F47BC4C1
:107BF0007B030000535745202020202020202020F8
:107C000020204F4E000C7CDC7B04000053574520A5
:107C10002020202020202020204F464600247CF4D5
:107C20007B84000053574620202020202020202045
:107C300020204F4E003C7C0C7C0500005357462012
:107C40002020202020202020204F464600547C2445
:107C50007C85000053574720202020202020202012
:107C600020204F4E006C7C3C7C0600005357472080
:107C70002020202020202020204F464600847C54B5
:107C80007C860000535748202020202020202020E0
:107C900020204F4E009C7C6C7C07000053574820EE
:107CA0002020202020202020204F464600B47C8425
:107CB0007C8700005357492020202020202020507E
:107CC0005245535300CC7C9C7C890000535749207B
:107CD000202020202052454C4541534500E47CB4EF
:107CE0007C09000053574A202020202020202020FB
:107CF0002020204100FC7CCC7C8B000053574A2084
:107D000020202020202020202020204200147DE45C
:107D10007C4B000053574A20202020202020202088
:107D200020202043002C7DFC7C8C000053574B20EE
:107D3000202020202020202020204F4E00447D1491
:107D40007D0D000053574B20202020202020202094
:107D5000204F4646005C7D2C7D8D000053574C2003
:107D600020202020202020505245535300747D4471
:107D70007D8E000053574C20202020202052454C5F
:107D800045415345008C7D5C7D0E000053574D20CE
:107D900020202020202020505245535300A47D74E1
:107DA0007D8F000053574D20202020202052454C2D
:107DB0004541534500BC7D8C7D0F000041696C65D9
:107DC000726F6E202020202020204F4E00D47DA4F2
:107DD0007D30000041696C65726F6E20202020208C
:107DE000204F464600EC7DBC7DB00000456C6576BA
:107DF00061746F722020202020204F4E00047ED41A
:107E00007D310000456C657661746F722020202002
:107E1000204F4646001C7EEC7DB100005275646424
:107E2000657220202020202020204F4E00347E0428
:107E30007E3200005275646465722020202020206C
:107E4000204F4646004C7E1C7EB200005468726F84
:107E500074746C652020202020204F4E00647E34F6
:107E60007E3300005468726F74746C65202020208B
:107E7000204F464600047B4C7EB30000202020416A
:107E800075746F20205472696D20202000967EA0AA
:107E90007F09803081005265736574204175746F6D
:107EA000205472696D7300B47E7C7E038CDB00828B
:107EB00068F25C002020205472696D20205A65729F
:107EC0006F20202000D27E967E038CDB0094680217
:107ED0005D00436C656172205472696D205A657251
:107EE0006F7300F07EB47E038CDB00A668525D00E9
:107EF00020416C7420202041697263726166742095
:107F0000000A7FD27E0980BA7F0020436F707920FB
:107F100020416972637261667420002A7FF07E05D9
:107F20008EDD00CA68765D685D0020205365742090
:107F300044656661756C7473202000487F0A7F0376
:107F40008CDB008268645E004E756D202070726F5D
:107F50007020626C6164657300687F2A7F05C8A524
:107F600003DC68010005000052657472616374737C
:107F7000205761726E696E6700847F487F0388A610
:107F800003706800204155584F555420436F6E745C
:107F9000726F6C2000A07F687F0080EC81BA0200C5
:107FA0004558495420202020202020202020202017
:107FB000007C7E847F0300CD000020416C74202370
:107FC0003120202020202020202000DA7F1681056B
:107FD00040CF030000000060000020416C742020AE
:107FE0002331205377697463682000F47FBA7F06D9
:107FF00080CE030020416C742023322020202020DA
:1080000020202020001480DA7F0540D103000000EA
:108010000060000020416C742020233220537769D7
:1080200074636820002E80F47F0680D00300204116
:108030006C74202333202020202020202020004E7C
:108040008014800540D30300000000600000204140
:108050006C74202023332053776974636820006890
:10806000802E800680D2030020416C7420233420AF
:1080700020202020202020200088804E800540D510
:10808000030000000060000020416C7420202334B5
:10809000205377697463682000A28068800680D4CA
:1080A000030020416C742023352020202020202034
:1080B000202000C28088800540D7030000000060B7
:1080C000000020416C7420202335205377697463AD
:1080D000682000DC80A2800680D6030020416C74FA
:1080E00020233620202020202020202000FC80C2B9
:1080F000800540D9030000000060000020416C743E
:10810000202023362053776974636820001681DCB1
:10811000800680D803004558495420202020202084
:1081200020202020202000BA7FFC800300CD00000A
:108130004154206D6F6465202020202020202020C5
:10814000004C819E810000B881B60200415420732A
:10815000746570202020202020202020006681309F
:108160008105009E02004154207469636B732020D6
:108170002020202020200080814C8105009F0200CB
:10818000746F20545A2020202020202020202020DE
:10819000009E8166810304DB000000A25D0045585B
:1081A0004954202020202020202020202020003082
:1081B0008180810300CD00004154206D6F646520F3
:1081C0002020202020496E6300D281D2810000B699
:1081D00002004154206D6F6465204F6E6520536826
:1081E0006F7400B881B8810100B602002020202001
:1081F000202020434831202020202020000482AC71
:10820000820100002020202020202043483220200E
:1082100020202020001C82EC810300002020202050
:1082200020202043483320202020202000348204B6
:1082300082050000202020202020204348342020D8
:1082400020202020004C821C8207000020202020BB
:108250002020204348352020202020200064823424
:1082600082090000202020202020204348362020A2
:1082700020202020007C824C820B00002020202027
:108280002020204348372020202020200094826492
:10829000820D00002020202020202043483820206C
:1082A0002020202000AC827C820F00002020202093
:1082B00020202050504D20202020202000EC8194B0
:1082C0008280000020202042756464792020426F63
:1082D0007820202000DE82F882098012830020208E
:1082E0002020205461626C6573202020202000F83B
:1082F00082C4820980AC8300455849542020202044
:10830000202020202020202000C482DE820300CDF7
:1083100000004D6173746572203F202020202020D2
:108320002020002C8362830300A1020020204D61E5
:108330007374657220204D6F64652020004883129D
:108340008300007C83B7020053747564656E7420EB
:108350003F202020202020200062832C830300A0C7
:108360000200455849542020202020202020202091
:10837000202000128348830300CD00004D204D6F64
:1083800064653D4D6963726F5374617200948394A8
:10839000830000004D204D6F64653D467574616239
:1083A00061202020007C837C83010000416972638E
:1083B00072616674205461626C65203100CC83EC7C
:1083C0008409860685DA03705E765E004169726311
:1083D00072616674205461626C65203200EC83AC7B
:1083E0008309860685E503705E765E00476C6F62E2
:1083F000616C20205461626C65202031000C84CCBB
:1084000083098606854602705E765E00476C6F6261
:10841000616C20205461626C65202032002C84EC59
:1084200083098606855102705E765E00476C6F6236
:10843000616C20205461626C65202033004C840CF8
:1084400084098606855C02705E765E00476C6F620A
:10845000616C20205461626C65202034006C842C97
:1084600084098606856702705E765E00476C6F62DF
:10847000616C20205461626C65202035008C844C36
:1084800084098606857202705E765E00476C6F62B4
:10849000616C20205461626C6520203600AC846CD5
:1084A00084098606857D02705E765E00476C6F6289
:1084B000616C20205461626C6520203700CC848C74
:1084C00084098606858802705E765E00476C6F625E
:1084D000616C20205461626C6520203800EC84AC13
:1084E00084098606859302705E765E00455849547D
:1084F00020202020202020202020202000AC83CC01
:10850000840300CD0000504F532030202020202035
:1085100020202020202000208524860100D000007B
:10852000504F5320312020202020202020202020A8
:10853000003A8506850100D10000504F53203220BB
:10854000202020202020202020200054852085016C
:1085500000D20000504F5320332020202020202024
:1085600020202020006E853A850100D30000504F66
:10857000532034202020202020202020202000886C
:108580008554850100D40000504F53203520202011
:10859000202020202020202000A2856E850100D5EB
:1085A0000000504F53203620202020202020202063
:1085B000202000BC8588850100D60000504F532044
:1085C00037202020202020202020202000D685A217
:1085D000850100D70000504F532038202020202054
:1085E00020202020202000F085BC850100D800003C
:1085F000504F5320392020202020202020202020D0
:10860000000A86D6850100D90000504F5320313032
:1086100020202020202020202020002486F08501FA
:1086200000DA000045584954202020202020202036
:10863000202020200006850A860300CD000020545B
:108640005820566F6C7420204D6574657220005A56
:1086500086DC870788C45E006900545820416C613D
:10866000726D20566F6C74616765007A863E86086D
:10867000C8B90200690000FF0000526573657420EC
:10868000426174742054696D65720098865A86033D
:108690008CDB008268FC5E0020525820566F6C74A0
:1086A00020204D657465722000B4867A860788E0C4
:1086B0005E006900536572766F20204D696E205010
:1086C000756C736500D486988602C8AE021269E89C
:1086D00003881300536572766F20204D6178205017
:1086E000756C736500F486B48602C8B0021269E83E
:1086F000038813004E756D62657220204368616EB9
:108700006E656C73001887D48605CEA202246904B6
:10871000000900A85EB05E0020202053796E63201F
:108720007769647468202020003887F48602C8A323
:10873000021269C800DC05002020536869667420B5
:10874000496E76657274202000548718870388CD9F
:10875000033669002020466F726D617420466C619B
:1087600073682020006E87388707800E5F00202006
:108770002020436F6E66696775726520202000882F
:10878000875487098056880020204A6F795374697E
:10879000636B2043616C202000A2876E87098012E2
:1087A0008B0020202020202020464D5320202020F8
:1087B000202000C0878887038CE9007068B85E00BD
:1087C000204672657175656E63792042616E642022
:1087D00000DC87A2870080F687D102004558495403
:1087E000202020202020202020202020003E86C085
:1087F000870300CD000020202020204E6F20205233
:10880000462020202020000E883E880000002020E6
:10881000202020353020204D487A2020202000269E
:1088200088F6870100002020202020353320204DAD
:10883000487A20202020003E880E88020000202058
:10884000202020373220204D487A2020202000F69A
:108850008726880300004F75747075742063686103
:108860006E6E656C2031007288A6890001C0890097
:1088700004004F7574707574206368616E6E656C6A
:108880002032008E8856880001C0890104004F758F
:1088900074707574206368616E6E656C203300AA15
:1088A0008872880001C0890204004F757470757465
:1088B000206368616E6E656C203400C6888E880007
:1088C00001C0890304004F7574707574206368617A
:1088D0006E6E656C203500E288AA880001C08904AC
:1088E00004004F7574707574206368616E6E656CFA
:1088F000203600FE88C6880001C0890504004F7537
:1089000074707574206368616E6E656C2037001A30
:1089100089E2880001C0890604004F75747075747F
:10892000206368616E6E656C2038003689FE8800B1
:1089300001C08907040053656C6563742041696C4C
:1089400020205472696D0052891A890001908AB200
:10895000020053656C65637420456C652020547279
:10896000696D006E8936890001908AB302005365F3
:108970006C6563742052756420205472696D008A9E
:108980008952890001908AB4020053656C65637452
:108990002054687420205472696D00A6896E890085
:1089A00001908AB5020045584954202020202020FB
:1089B0002020202020200056888A890300CD000036
:1089C0002020202041696C65726F6E2020202020BD
:1089D00000DA89768A0100DC000020202020456C26
:1089E000657661746F722020202000F489C08902AE
:1089F00000DC000020202020205275646465722075
:108A000020202020000E8ADA890300DC00002020CC
:108A100020205468726F74746C6520202020002818
:108A20008AF4890400DC000020202020202020433C
:108A3000483520202020202000428A0E8A0500DCB4
:108A40000000202020202020204348362020202005
:108A50002020005C8A288A0600DC000020202020DC
:108A600020202043483720202020202000768A42E2
:108A70008A0700DC000020202020202020434838E6
:108A800020202020202000C0895C8A0800DC000013
:108A9000202020204E6F20205472696D202020203D
:108AA00000AA8AF88A0000DC000020202020205440
:108AB00072696D2031202020202000C48A908A0114
:108AC00000DC000020202020205472696D2032201C
:108AD0002020202000DE8AAA8A0200DC000020205C
:108AE0002020205472696D2033202020202000F89F
:108AF0008AC48A0300DC00002020202020547269F0
:108B00006D2034202020202000908ADE8A0400DCA2
:108B100000002020202041696C65726F6E202020AB
:108B20002020002E8B2A8C0780CE60150400202088
:108B30002020456C657661746F7220202020004AE9
:108B40008B128B0780CE601B0500202020205275E1
:108B50006464657220202020202000668B2E8B0705
:108B600080CE60210600202020205468726F74742B
:108B70006C652020202000828B4A8B0780006027B4
:108B800007002020202020204348362020202020BD
:108B90002020009E8B668B0780145F3B0000202006
:108BA000202020204348372020202020202000BAE9
:108BB0008B828B0780145F3F0100202041696C6528
:108BC000726F6E207472696D202000D68B9E8B07A9
:108BD00080145F2B080020456C657661746F7220ED
:108BE000207472696D2000F28BBA8B0780145F2F9E
:108BF0000900202052756464657220207472696DCA
:108C00002020000E8CD68B0780145F330A0020547E
:108C100068726F74746C6520207472696D20002A0C
:108C20008CF28B0780145F370B0045786974202025
:108C30002020202020202020202000128B0E8C03BA
:108C400000CD00002020202043656E746572202036
:108C500020202020000020202052696768742F44C3
:108C60006F776E2020200000202020204C65667445
:108C70002F55702020202020000001000F00D2007E
:108C800000000300D20000001E00D2000080121B72
:108C900001660379013C012E03AE01130126039501
:108CA0000162017300860412018B040701C80405E8
:108CB000012A042901320237023B022F0200000878
:108CC0000001040910192431405164001324334079
:108CD0004B545B60636400010203060C15223349A8
:108CE00064001B31424F585E61626364000A141EC7
:108CF00028323C46505A640014283C5064503C28AA
:108D0000140000050A0F14192837465564000F1E79
:108D10002D3C4B50555A5F640A0A0000109001FF29
:108D200000A5E7C009F30000DC059411010203046B
:108D30000000FF5801000102830405060708090A24
:108D40000B8C8D0E0F0000000000000000000000E2
:108D50000000000000000000000000000000000013
:108D60000000000000000000000000000000000003
:108D7000000000000000000000004D4F44454C2062
:108D800030312020202020202020000001B80B00BE
:108D9000013C190000000001B80B00013C19000063
:108DA000000001B80B00013C1900000000FEA00FFC
:108DB0001901D0070001B80B0001B80B0001B80B76
:108DC0000001B80B000132FF320032003200CEFF4A
:108DD000CE00CE00CE0000000014140000000A0AED
:108DE0000000000A0A0000000A0A0000F4010A005C
:108DF00000000A0A0000000A0A0000000A0A000037
:108E0000000A0A0000000A0A0000000A0A00000026
:108E10000A0A000000000000000A00000000000232
:108E200000000000000000FF0001028304050607A7
:108E3000898B4B8C0D8E8F0100081000074B8C0422
:108E400000200000000000FF0D0020002000200096
:108E50002000200000010409101924314051640051
:108E6000132433404B545B60636400000000000037
:108E700000000000000000000000020103040506DD
:108E800007080000000000000000000000000000D3
:108E900000000000000000000000000000000000D2
:108EA00000000000000000000000000000000000C2
:108EB00000000000000000000000000000000000B2
:108EC00000000000000000000000000000000000A2
:108ED0000000000000000000000000000000000092
:108EE0000000000000000000000000000000000082
:108EF0000000000000000000000000000000000072
:108F00000000000000000000000000000000000061
:108F10000000000000000000000000000000000051
:108F20000000000000000000000000000000000041
:108F30000000000000000000000000000000000031
:108F40000000000000000000000000000000000021
:108F50000000000000000000000000000000000011
:108F60000000000000000000000000000000000001
:0A8F700000000000000000000000F7
:00000001FF
